:0400000057EF00F0C6
:100008002B002B002B002B002B002B002B002B0090
:10001800085D2B002B002B002B002B002B002B0046
:100028002B002B002B002B002B002B002B002B0070
:100038002B002B002B006A592B002B002B002B00C8
:100048002B002B002B002B002B002B002B002B0050
:100058002B002B002B002B002B002B002B002B0040
:100068002B002B002B002B002B002B002B002B0030
:10007800825E2B002B002B002B002B002B002B006B
:100088002B002B002B002B002B002B002B002B0010
:100098002B002B002B002B002B002B002B002B0000
:0A00A8002B002B00FF0030EFB1F039
:10F3EA000000000000001B1B0000181818181B1B47
:10F3FA000000030303031B1B00001B1B1B1B1B1B1F
:10F40A0000040E1F0404040400040404041F0E0470
:10F41A00001F1F1F1F1F1F1F000E0A0E00000000E3
:10F42A00002C7C01B27801427B01E254014866015A
:10F43A00A269010265011E7C01CA7C01C67C01BA6F
:10F44A007901727C017A7C01107C016A7C01007C62
:10F45A0001C86D018C6B01F07B010024744C0024FF
:10F46A00744C0000FA460024F4480000FA46008072
:10F47A00C094D43F358640202000204469726563D9
:10F48A00746F7279203A433A5C4D504C4142585F4E
:10F49A0050726F6A656374735C5F31384632374BFA
:10F4AA0034325F494E413232365F4932435F4C4310
:10F4BA00445F554152545F323032352E580D0A009E
:10F4CA002052423020696E3D414C457274202C20F6
:10F4DA005241343D6C65642C2052433250505320C3
:10F4EA004E434F31206F75743D42757A7A65722C9E
:10F4FA0055415254205243363D54582C5243373DBD
:10F50A0052580D0A002050494331384632374B349D
:10F51A0032202B205465737420494E4132323620F2
:10F52A0052313030204932432073656E736F722036
:10F53A000D0A20456E204D6F6465204443205057C4
:10F54A004D20344B687A0D0A0045434F2E2E2E2E3D
:10F55A000042415252455F470042415252455F4480
:10F56A00004241525245474400464C4543482048D0
:10F57A0000464C4543485F42004E4F49522E2E2EBC
:10F58A000044454752454320002054657374205077
:10F59A00574D3520313020626974732D3E52433104
:10F5AA00707073204F75742D3E204D4F534645544D
:10F5BA002D3E416D706F756C65203132562035775E
:10F5CA000D0A0020496E636C7564653A202044690F
:10F5DA00616C6F6775655F4F70657261746575728E
:10F5EA005F50435F7669615F554152545F323032F2
:10F5FA00352D30322E696E630D0A00204C434420AB
:10F60A0034783230206361727320737572206275A8
:10F61A00732049324331204857203A205243333D20
:10F62A0053434C2C5243343D5344410D0A0020505D
:10F63A00726F6A656374203A20205F313846323728
:10F64A004B34325F4932435F4C435F554152545FFA
:10F65A00323032330D0A002041696775696C6C617A
:10F66A00676520736F7274696520766961205243F9
:10F67A00315050533D2030783044200020436F6E83
:10F68A006669672020496E7465726E616C20466FE8
:10F69A0073632036344D487A0D0A0020536F757211
:10F6AA006365203A20206D61696E2E63205F3230D7
:10F6BA0032352D303232370D0A0020204D46494E60
:10F6CA00544F53432028353030206B487A29002084
:10F6DA004D46494E544F53432F3420283332206B22
:10F6EA00487A2900202020202020202020202020A5
:10F6FA00202020202020202000204846494E544F18
:10F70A0053432000204C46494E544F534300204651
:10F71A004F53430020416C61726D65207669612008
:10F72A00696E74657272757074696F6E203A2073AF
:10F73A006F7274696520414C4552544520494E41C7
:10F74A00323236202D3E2052423020696E70757456
:10F75A00200D0A004D4F4445202052616D706520EE
:10F76A003A20204D4F443D312073696E6F6E204D13
:10F77A004F443D30203D3E757361676520646520C6
:10F78A00436F6E7369676E655F447574795F50572E
:10F79A004D0D0A000D0A202052616D706520444FFC
:10F7AA00574E2020203130323420E02030206D6145
:10F7BA00697320636865636B2073757220696E7460
:10F7CA00657276616C206465203332207061730D36
:10F7DA000A000D0A2052616D7065202055502030B4
:10F7EA0020E02031303234202C6D61697320636847
:10F7FA0065636B2073757220696E74657276616CCD
:10F80A0020646520333220706173200D0A0046722D
:10F81A0065712050574D353D7820617665632031FA
:10F82A003D33324B687A202E2E2E20323D31364B14
:10F83A00687A2E2E20333D384B687A202E2E2E20C1
:10F84A00373D353030487A0D0A0020416C657274B4
:10F85A00204D41534B5F454E5F52454720726567C5
:10F86A00697374657220303768203C2D2031302E40
:10F87A0030303020706F7572203235306D410D0A8C
:10F88A000020436F6D70696C65206C6520257320BC
:10F89A0061202573205554430D0A20617665632043
:10F8AA0076657273696F6E20584338203A20202596
:10F8BA0064200D0A0020415454454E54494F4E20AD
:10F8CA003A20416472657373652049324320204CA3
:10F8DA004344203478323020646566696E69652055
:10F8EA0064616E73203A0D0A002052656C65637478
:10F8FA00757265202076616C657572206465204D8D
:10F90A0041534B5F454E5F524547207265676973A5
:10F91A0074657220303768200D0A00204D61736BC0
:10F92A002F416C65727420204D41534B5F454E5FE9
:10F93A00524547207265676973746572203036686C
:10F94A00203C2D203078383030310D0A00204368B1
:10F95A00617267656D656E74206361726163746557
:10F96A007265732053706563696175782073657475
:10F97A0020233120656E20434752414D0D0A002055
:10F98A0053617576652076616C6575722064616E67
:10F99A007320204D41534B5F454E5F5245472072BD
:10F9AA006567697374657220303768200D0A002014
:10F9BA00436F6E6669672020494E413232365F4393
:10F9CA004F4E465F5245472C3078343346462028FE
:10F9DA007761732030783431323720290D0A0020BC
:10F9EA000D0A53657175656E6365206427496E69F2
:10F9FA0074204C434420347832302076696120499F
:10FA0A0032433120504346383537340D0A002049F5
:10FA1A006E69742050574D352031302062697473F5
:10FA2A00202873757220524331292020467265714D
:10FA3A003D2025356420487A200D0A0020402064A4
:10FA4A006563696D616C20232534752020736F69A5
:10FA5A00742040446576696365203762697473204F
:10FA6A003D203058253032582000536575696C2086
:10FA7A00616C61726D6520636F757272616E74205C
:10FA8A00656E206D4120533D30313020E020383101
:10FA9A0039200D0A00436F6E7369676E655F44759E
:10FAAA0074795F50574D203A20434F4E533D3030C2
:10FABA00303120E02031303233200D0A00204361FA
:10FACA006C6962726174696F6E20726567697374BA
:10FADA00657220303568203C2D2030783030333440
:10FAEA00200D0A000D0A204E6F7576656C6C652034
:10FAFA00436F6E7369676E65204475747920505739
:10FB0A004D203D20253035640D0A0020546573745C
:10FB1A002070726573656E636520646576696365D6
:10FB2A0073207375722042757320493243310D0A6E
:10FB3A00002046696E20646520706172616D65748B
:10FB4A007261676520494E413232362E2E2E204F81
:10FB5A004B0D0A0D0A0020766961206C69676E6593
:10FB6A002023646566696E65204C43445F414444C2
:10FB7A00522030787878200D0A000D0A20496E69E3
:10FB8A00745F54696D657232282920286173736F16
:10FB9A006369E920E02050574D35290D0A00204EAF
:10FBAA00455720536575696C206427616C657274CA
:10FBBA00652025332E336620416D70657265730D9D
:10FBCA000A0020426F75636C65207072696E636902
:10FBDA0070616C65202070726F6772616D6D65204F
:10FBEA000D0A002030783237206176656320507222
:10FBFA006F746F20426173652031384632374B3457
:10FC0A00320D0A002061647265737365204C4344A7
:10FC1A003D20256420736F6974203058253032588E
:10FC2A00200D0A0020546573742042757A7A657231
:10FC3A002073757220736F72746965205243322083
:10FC4A000D0A00204D657375726520646520636F27
:10FC5A007572616E742025203564206D41200D0A6D
:10FC6A0000206572722073757220636F6E73696704
:10FC7A006E6520447574792050574D0D0A00204C4A
:10FC8A0043445F34626974735F4932435F3230328E
:10FC9A00332D303831302E680D0A0020434B505333
:10FCAA003D203078253032582020467265713D2536
:10FCBA00356420487A0D0A00456570726F6D2032EE
:10FCCA00344C43787878203235366B206F7520357E
:10FCDA0031324B002041666669636861676520734B
:10FCEA007572204C43442034783230200D0A0020AB
:10FCFA00494E41204D616E75666163747565722067
:10FD0A00203078253034580D0A0020544D523420C2
:10FD1A00696E697469616C697365202831736563FA
:10FD2A00290D0A00252033642020456E20636F7553
:10FD3A007273203A25203564206D410D0A0020494E
:10FD4A004E41204964656E74696669616E7420303B
:10FD5A0078253034580D0A00205043463837353458
:10FD6A0020666F72204C43442032783136636172C8
:10FD7A00730020496E69745F493243282920E020C4
:10FD8A003130304B687A3B0D0A002025332E33661A
:10FD9A0020572020536575696C3D25332E33662024
:10FDAA0041002050574D352044757479203D202557
:10FDBA003464202563200D0A0020494E4132323630
:10FDCA005F496E69745F436F6E666967200D0A004A
:10FDDA000D0A2048656C7020436F6D6D616E646515
:10FDEA0073203A0D0A0020496E6974204E434F3140
:10FDFA0020E02031303030487A0D0A002025332E99
:10FE0A0032662056202025332E33662041202020BA
:10FE1A002000494E413232362054657374732032C1
:10FE2A003032353032323700494E41323236204391
:10FE3A00757272656E742073656E736F72002056E8
:10FE4A00657273696F6E2050726F6772616D6D654E
:10FE5A0020200031323334353637383930313233B5
:10FE6A0034353637383930004361726163746572EC
:10FE7A006573205370656369617578320041424346
:10FE8A004445464748494A4B4C4D4E4F50515253B0
:10FE9A005400202025322E33662056202025322E6B
:10FEAA00336620412000206D76413D2520356420AF
:10FEBA006D76553D252035642000323032352D309F
:10FECA003232372031384632374B343200504346CB
:10FEDA00383537344120386269747320492F4F000E
:10FEEA00204E6220626F75636C65733D2535642010
:10FEFA0020004C4344203231313920327831366384
:10FF0A006172730050434638353734203862697459
:10FF1A007320494F00204D6F64652052616D7065F2
:10FF2A003D300D0A00252033642020252035642029
:10FF3A006D410D0A002050726573656E74617469B3
:10FF4A006F6E203A0020553D252035642020413D22
:10FF5A002520356400454550524F4D2035313262D7
:10FF6A007974657300736575696C206B3D2025355E
:10FF7A00642020004D6F64652052616D7065203DDC
:10FF8A0020004F4C4544205353443133303600252A
:10FF9A003564204146463D256420006E6F6E20631D
:10FFAA006F6E6E752021004665622032372032302E
:10FFBA0032350020493D253564206D4120005254D8
:10FFCA0043204453333233310031373A30373A35EC
:10FFDA00310052656375203A00494E46004E414E43
:10FFEA0000696E66006E616E006C6C7300202E31C3
:05FFFA00006C66000030
:020000040001F9
:10000000600E3901D96F000EDB6F000EDD6F080E38
:10001000DF6F000EDE6F090E0001EA6F1E0EE96F42
:10002000E40EE82EFED7E92FFCD7EA2FFAD700F02E
:10003000000E3901C26F000EC36F4DECAFF0D29EBF
:100040003901909F000E3A01456F000E466F000E79
:10005000476F000E656F000E666F000E676F000E33
:10006000556F000E566F010E866F000E556F010E14
:10007000566F000E576FD2903901909F9181A09FCB
:10008000A191000E0001F86F000EF76F000EF7252A
:10009000D96E030EF821DA6E000EDF6EF74BF82BE7
:1000A000F85109E1800EF75DD8A059EF80F05BEFC1
:1000B00080F046EF80F0000EF86F000EF76F800EB4
:1000C000F725D96E030EF821DA6E000EDF6EF74BBE
:1000D000F82BF85109E1800EF75DD8A072EF80F09F
:1000E00074EF80F05FEF80F0000EF86F000EF76F96
:1000F000700EF725D96E020EF821DA6E000EDF6E53
:10010000F74BF82BF85109E14F0EF75DD8A08BEFB4
:1001100080F08DEF80F078EF80F0000EF36F030E2B
:10012000F46F83ECB9F0090E0001EA6F1E0EE96F5F
:10013000E40EE82EFED7E92FFCD7EA2FFAD700F01D
:100140002BECBCF02BECBCF03F0E036EFF0E046EEC
:1001500039ECB8F02BECBCF0000E0001F86F000E8B
:10016000F76FD890F735D96EF835DA6EC00ED9260C
:10017000020EDA226F0078FF03F06F0074FF04F0C4
:1001800039ECB8F0BA78090E0001EA6F1E0EE96F7B
:10019000E40EE82EFED7E92FFCD7EA2FFAD700F0BD
:1001A0000001F74BF82BF85109E1090EF75DD8A0D3
:1001B000DCEF80F0DEEF80F0B1EF80F02BECBCF0F4
:1001C000F3C0C9F0F4C0CAF08B0E0001CB6FF80E7B
:1001D000CC6FB10ECD6FFF0ECE6FD30ECF6FFF0E73
:1001E000D06F090ED26F380ED16FB7ECB8F0F3C0F4
:1001F00003F0F4C004F0ACECB6F02BECBCF0F00E65
:10020000036EFD0E046E39ECB8F010ECB5F02E0E56
:10021000036EFC0E046E39ECB8F0090E0001EA6FB3
:100220001E0EE96FE40EE82EFED7E92FFCD7EA2F69
:10023000FAD700F03F013E9F090E0001EA6F1E0E43
:10024000E96FE40EE82EFED7E92FFCD7EA2FFAD7A4
:1002500000F03F013E8F110E0001EA6F3C0EE96F86
:10026000CB0EE82EFED7E92FFCD7EA2FFAD73F01B5
:100270003E9F2BECBCF07C0E036EFD0E046E39EC41
:10028000B8F017ECBDF0150E036EFB0E046E39ECE2
:10029000B8F063EC9FF02BECBCF0270E0001FA6F76
:1002A000BF0E036EF80E046E39ECB8F0880E036EC4
:1002B000FC0E046E39ECB8F0600E036EFB0E046E9B
:1002C00039ECB8F0ED0E036EFB0E046E39ECB8F0AD
:1002D0002BECBCF0000E0001FF6F140EFE6F270E1A
:1002E000FA6F700EC96F020ECA6F0E0ECB6FFC0E46
:1002F000CC6FFAC0CDF0CE6BFAC0CFF0D06BB7ECBC
:10030000B8F0700E036E020E046EACECB6F0E90E9F
:10031000036EF90E046E39ECB8F0D3ECA9F02BECB7
:10032000BCF0010E4AECB4F0090E0001EA6F1E0E9B
:10033000E96FE40EE82EFED7E92FFCD7EA2FFAD7B3
:1003400000F0020E4AECB4F0090E0001EA6F1E0E36
:10035000E96FE40EE82EFED7E92FFCD7EA2FFAD793
:1003600000F0DE0E036EFC0E046E39ECB8F0870E62
:10037000216EFE0E226E4EECB5F0000E276E020EC0
:10038000266EB2ECAFF05D0E216EFE0E226E4EECCC
:10039000B5F0000E276E030E266EB2ECAFF0480EDD
:1003A000216EFE0E226E4EECB5F0000E276E040E8E
:1003B000266EB2ECAFF0C40E216EFE0E226E4EEC35
:1003C000B5F0020E64ECB8F0000E0001F86F000EFC
:1003D000F76F570E036EF90E046E39ECB8F0010E8C
:1003E0004AECB4F0D00E0001E96FC90EE82EFED73A
:1003F000E92FFCD700D0000E276E010E266EB2EC5E
:10040000AFF0720E216EFE0E226E4EECB5F0000EB5
:10041000276E020E266EB2ECAFF0D00E0001E96F2F
:10042000C90EE82EFED7E92FFCD700D0000E236EB0
:10043000000E226E34ECA9F0840E036EFB0E046EE7
:1004400039ECB8F077ECBAF0700E0001C96F020E0B
:10045000CA6F180ECB6FFA0ECC6FD8900101E93538
:10046000D96EEA35DA6EC80ED926010EDA226F008F
:1004700078FFCDF06F0074FFCEF0B7ECB8F0700EDF
:10048000036E020E046EACECB6F095ECBDF0000EFF
:100490000101676F960E666F1F0E036EFF0E046EEE
:1004A00039ECB8F066C103F067C104F099ECBBF019
:1004B00066C103F067C104F0000E066E0A0E056EF9
:1004C00015ECB0F003C0F7F104C0F8F1700E0001B4
:1004D000C96F020ECA6FAC0ECB6FFD0ECC6FF7C1A9
:1004E000CDF0F8C1CEF0000ED06F250ECF6FB7EC77
:1004F000B8F0700E036E020E046EACECB6F02BEC8E
:10050000BCF0520E0001EA6F2B0EE96F000EE82ED0
:10051000FED7E92FFCD7EA2FFAD700F02BECBCF07E
:10052000000E0101736F000E726F000E716F000EEE
:10053000706FC30E036EFD0E046E39ECB8F097ECCD
:1005400099F0CC0E036EFB0E046E39ECB8F01E0E63
:10055000036EF70E046E39ECB8F050ECB7F03901C9
:10056000A191A7919181D28E140E036EFD0E046E9F
:1005700039ECB8F0D5ECBAF0000E0101816F000E35
:10058000806F2BECBCF08BECB5F014EC9EF0270EDA
:100590000001FA6F04ECABF014EC9EF0AAECA0F0B2
:1005A000010164056511D8A4D8EF82F0DAEF82F07A
:1005B000EFEF82F0DC0E036EF70E046E39ECB8F04C
:1005C000010EC3ECA3F09E0E036EF70E046E39EC21
:1005D000B8F0000EC3ECA3F0BA8802EF83F066C156
:1005E00003F067C104F099ECBBF0520E0001EA6F12
:1005F0002B0EE96F000EE82EFED7E92FFCD7EA2F6D
:10060000FAD700F00101B305D8A409EF83F00BEF8E
:1006100083F04FEF87F0DC0E036EFF0E046E39ECB3
:10062000B8F0800E0001F16F030EF26FF1C003F01D
:10063000F2C004F0ACECB6F02BECBCF06000C7F3F9
:10064000D9FF6000CBF3DAFF480EDE18D8A42BEFF9
:1006500083F02DEF83F080EF83F0000120EE01F0B6
:10066000F151D926F251DA22650EDE18D8A43BEFFB
:1006700083F03DEF83F080EF83F020EE02F0F15144
:10068000D926F251DA226C0EDE18D8A44AEF83F094
:100690004CEF83F080EF83F020EE03F0F151D92688
:1006A000F251DA22700EDE18D8A459EF83F05BEF16
:1006B00083F080EF83F0DA0E036EFD0E046E39ECEA
:1006C000B8F0740E036EFA0E046E39ECB8F0180E22
:1006D000036EF80E046E39ECB8F09F0E036EFA0E3E
:1006E000046E39ECB8F05E0E036EF70E046E39EC52
:1006F000B8F02BECBCF0000E0001F16F000EF26FB1
:100700006000C7F3D9FF6000CBF3DAFF530EDE18A9
:10071000D8A48DEF83F08FEF83F0C9EF84F0000150
:1007200020EE01F0F151D926F251DA223D0EDE1809
:10073000D8A49DEF83F09FEF83F0C9EF84F0F1C060
:1007400003F0F2C004F00DECB8F0050E031804102D
:10075000D8A4ADEF83F0AFEF83F0C9EF84F00001D0
:1007600020EE02F0F151D926F251DA22DF50D00FFB
:10077000FB6FFB51640D6F00CCFFFCF06F00D0FFEE
:10078000FDF020EE03F0F151D926F251DA22DF50CC
:10079000D00FFB6FFB510A0D6F00CCFFE9F06F002B
:1007A000D0FFEAF0FC51E925FC6FFD51EA21FD6F15
:1007B00020EE04F0F151D926F251DA22DF50D00FA9
:1007C000FB6FFB51FC25FC6F000EFD21FD6FFD5101
:1007D00009E10A0EFC5DD8A0F0EF83F0F2EF83F0A0
:1007E000C4EF84F0340EFC5D030EFD59D8B0FBEF6E
:1007F00083F0FDEF83F0C4EF84F0FCC003F0FDC094
:1008000004F0000E066E280E056EB3ECBCF003C0BB
:10081000FCF004C0FDF0700E0001C96F020ECA6F3B
:100820006F0ECB6FFF0ECC6FFCC0CDF0FDC0CEF0D5
:10083000B7ECB8F0700E036E020E046EACECB6F0BE
:1008400039019191890E036EF90E046E39ECB8F0FE
:10085000070E0101B46F0001FD510101B56FFCC02D
:10086000B6F1400E0001FA6FB40EEF6F010EF06F9B
:10087000030EFB6FEFC018F0F0C019F0FBC01AF0C8
:100880001B6AFA51B0ECB7F0F30E036EF80E046E6B
:1008900039ECB8F0400E0001FA6F000E0101B46FA0
:1008A000000EB56FB40E0001EF6F010EF06F070E72
:1008B000186EEFC019F0F0C01AF0000E1C6E030E97
:1008C0001B6EFA518EECB4F00101B4510001EA6FD5
:1008D000E96B0101B5510001E925FC6F0101000E32
:1008E0000001EA21FD6F170E156EB70E166E510E40
:1008F000176E3F0E186EFCC003F0FDC004F0056AD1
:10090000066A000EAAECA4F003C011F004C012F0B5
:1009100005C013F006C014F0A3EC95F011C02AF046
:1009200012C02BF013C02CF014C02DF0000E2E6E50
:10093000000E2F6E000E306E470E316ECAEC97F02F
:100940002AC03AF12BC03BF12CC03CF12DC03DF147
:10095000700E0001C96F020ECA6FA80ECB6FFB0E9E
:10096000CC6F3AC1CDF03BC1CEF03CC1CFF03DC120
:10097000D0F0B7ECB8F0700E036E020E046EACEC63
:10098000B6F03901A1919181000E0001F16F000EC6
:10099000F26F6000C7F3D9FF6000CBF3DAFF500EAF
:1009A000DE18D8A4D6EF84F0D8EF84F072EF85F08B
:1009B000000120EE01F0F151D926F251DA22570E52
:1009C000DE18D8A4E6EF84F0E8EF84F072EF85F04B
:1009D00020EE02F0F151D926F251DA224D0EDE1846
:1009E000D8A4F5EF84F0F7EF84F072EF85F020EEF5
:1009F00003F0F151D926F251DA223D0EDE18D8A4C7
:100A000004EF85F006EF85F072EF85F0F1C003F09A
:100A1000F2C004F00DECB8F0045009E1040E035CE0
:100A2000D8A015EF85F017EF85F072EF85F0000183
:100A300020EE04F0F151D926F251DA22DF50D00F26
:100A4000FB6FFB51D8B427EF85F029EF85F06DEFF0
:100A500085F0080EFB612FEF85F031EF85F06DEF2B
:100A600085F0FBC0E9F10101EA6BAC9E700E00015C
:100A7000C96F020ECA6FA50ECB6FFC0ECC6FFBC008
:100A8000CDF0CE6BD8900101E935D96EEA35DA6E3A
:100A9000C80ED926010EDA226F0078FFCFF06F0062
:100AA00074FFD0F0B7ECB8F0700E036E020E046E57
:100AB000ACECB6F00001FB39F00BFB6FAC500F0B48
:100AC000AC6EAC50FB11AC6EFA0EAB6E000EAA6EA3
:100AD0003901A495AC8E2BECBCF0000E0001F16F37
:100AE000000EF26F6000C7F3D9FF6000CBF3DAFFAE
:100AF0004D0EDE18D8A47FEF85F081EF85F0F0EF82
:100B000085F0000120EE01F0F151D926F251DA22F0
:100B10004F0EDE18D8A48FEF85F091EF85F0F0EF3F
:100B200085F020EE02F0F151D926F251DA22440E7E
:100B3000DE18D8A49EEF85F0A0EF85F0F0EF85F0E9
:100B400020EE03F0F151D926F251DA223D0EDE18E3
:100B5000D8A4ADEF85F0AFEF85F0F0EF85F0F1C0F0
:100B600003F0F2C004F00DECB8F0045009E1040EFB
:100B7000035CD8A0BEEF85F0C0EF85F0F0EF85F004
:100B8000000120EE04F0F151D926F251DA22DF50B3
:100B9000D00FFB6FFB05D8A4D0EF85F0D2EF85F026
:100BA000D9EF85F0000E0101656F010E646FDEEF75
:100BB00085F0000E0101656F000E646F7E0E036EFE
:100BC000FF0E046E39ECB8F001016451300F3BECBC
:100BD000BDF02BECBCF0000E0001F16F000EF26FC7
:100BE0006000C7F3D9FF6000CBF3DAFF430EDE18D5
:100BF000D8A4FDEF85F0FFEF85F04FEF87F00001FF
:100C000020EE01F0F151D926F251DA224F0EDE1812
:100C1000D8A40DEF86F00FEF86F04FEF87F020EEAF
:100C200002F0F151D926F251DA224E0EDE18D8A484
:100C30001CEF86F01EEF86F04FEF87F020EE03F0FA
:100C4000F151D926F251DA22530EDE18D8A42BEF37
:100C500086F02DEF86F04FEF87F020EE04F0F15193
:100C6000D926F251DA223D0EDE18D8A43AEF86F0EA
:100C70003CEF86F04FEF87F0F1C003F0F2C004F0D4
:100C80000DECB8F0045009E1090E035CD8A04BEF5D
:100C900086F04DEF86F04FEF87F0D00E0001E96F40
:100CA000FF0EEA6F20EE05F0F151D926F251DA225B
:100CB000DF50EB6FEC6BE951EB27EA51EC23EC5181
:100CC00007E10A0EEB5DD8B068EF86F06AEF86F0B8
:100CD00042EF87F0D00EE96FFF0EEA6F20EE06F0CC
:100CE000F151D926F251DA22DF50EB6FEC6BE9516A
:100CF000EB27EA51EC23EC5107E10A0EEB5DD8B08B
:100D000084EF86F086EF86F042EF87F0D00EE96F31
:100D1000FF0EEA6F20EE07F0F151D926F251DA22E8
:100D2000DF50EB6FEC6BE951EB27EA51EC23EC5110
:100D300007E10A0EEB5DD8B0A0EF86F0A2EF86F0D7
:100D400042EF87F0D00EE96FFF0EEA6F20EE08F059
:100D5000F151D926F251DA22DF50EB6FEC6BE951F9
:100D6000EB27EA51EC23EC5107E10A0EEB5DD8B01A
:100D7000BCEF86F0BEEF86F042EF87F0000EFD6F0D
:100D8000000EFC6F20EE05F0F151D926F251DA2267
:100D9000DF50D00FFB6FFBC003F0046A030E066E3A
:100DA000E80E056EB3ECBCF003C0FCF004C0FDF02F
:100DB000000120EE06F0F151D926F251DA22DF507F
:100DC000D00FFB6FFB51640D6F00CCFFE9F06F009B
:100DD000D0FFEAF0FC51E925FC6FFD51EA21FD6FDF
:100DE00020EE07F0F151D926F251DA22DF50D00F70
:100DF000FB6FFB510A0D6F00CCFFE9F06F00D0FFD5
:100E0000EAF0FC51E925FC6FFD51EA21FD6F20EE6F
:100E100008F0F151D926F251DA22DF50D00FFB6FE2
:100E2000FB51FC25FC6F000EFD21FD6FFC51FD11F7
:100E3000D8B41DEF87F01FEF87F048EF87F0040E5E
:100E4000FD5DD8B026EF87F028EF87F048EF87F0F8
:100E5000FCC066F1FDC067F1700EC96F020ECA6F6B
:100E6000EE0ECB6FFA0ECC6F66C1CDF067C1CEF03F
:100E7000B7ECB8F0700E036E020E046EACECB6F078
:100E800048EF87F06B0E036EFC0E046E39ECB8F081
:100E90002BECBCF0000E0001F16F000EF26F0101AF
:100EA000964B972BC3EF82F057EF00F0000E000136
:100EB0007C6F000E7B6F62C08DF063C08EF064C0EB
:100EC0008FF065C090F090BF6AEF87F068EF87F011
:100ED00080EF87F0000E7C6F010E7B6F8DC003F0FA
:100EE0008EC004F08FC005F090C006F047ECBBF058
:100EF00003C08DF004C08EF005C08FF006C090F0E6
:100F0000000E0001946F000E936F5CC17FF05DC115
:100F100080F07B517C11D8A490EF87F092EF87F09E
:100F200099EF87F05CA497EF87F099EF87F0B3EF24
:100F300087F07B517C11D8A4A0EF87F0A2EF87F057
:100F4000A8EF87F0000E686F2B0E676FACEF87F08D
:100F5000000E686F2D0E676F67C020F2934B942BC5
:100F60007F07D8A080078DC003F08EC004F08FC02B
:100F700005F090C006F017ECADF003040410D8A4FF
:100F8000C4EF87F0C6EF87F010EF88F0BF0E576E02
:100F9000FF0E586E00016651596E5A6A5750592615
:100FA00058505A225A5007E11A0E595CD8B0DBEF5C
:100FB00087F0DDEF87F0EBEF87F0200E9325076ECB
:100FC000020E9421086EE30E096EFF0E0A6E1BECF2
:100FD000B7F0F7EF87F0200E9325076E020E9421ED
:100FE000086EEB0E096EFF0E0A6E1BECB7F00001E7
:100FF000FD0E7F27FF0E802360C013F061C014F048
:10100000200E156E020E166E7FC017F080C018F00D
:1010100077ECB0F013C060F014C061F05DEF8DF0BC
:101020008DC003F08EC004F08FC005F090C006F0B4
:1010300017ECADF003500410D8A421EF88F023EF93
:1010400088F056EF88F0BF0E576EFF0E586E000105
:101050006651596E5A6A5750592658505A225A505A
:1010600007E11A0E595CD8B038EF88F03AEF88F0F3
:1010700048EF88F0200E9325076E020E9421086E2B
:10108000E70E096EFF0E0A6E1BECB7F0F7EF87F064
:10109000200E9325076E020E9421086EEF0E096E46
:1010A000FF0E0A6E1BECB7F0F7EF87F0000E0001A1
:1010B000956F000E966F800E976F3F0E986F000E23
:1010C000926F000E916F8DC003F08EC004F08FC040
:1010D00005F090C006F0000E076E000E086E000EC0
:1010E000096E000E0A6E87ECB1F0D8B07AEF88F086
:1010F0007CEF88F0FFEF88F09BEF88F095C011F04F
:1011000096C012F097C013F098C014F0000E156E40
:10111000000E166E200E176E410E186EA3EC95F0A1
:1011200011C095F012C096F013C097F014C098F05B
:101130000001914B922B8DC02AF08EC02BF08FC0F6
:101140002CF090C02DF0000E156E000E166E200EC5
:10115000176E410E186E95C011F096C012F097C030
:1011600013F098C014F0A3EC95F011C02EF012C04B
:101170002FF013C030F014C031F013ECACF0D8B045
:10118000C4EF88F0C6EF88F07EEF88F0E6EF88F0D5
:1011900095C02AF096C02BF097C02CF098C02DF087
:1011A000000E2E6E000E2F6E200E306E410E316E30
:1011B000CAEC97F02AC095F02BC096F02CC097F09F
:1011C0002DC098F000019107D8A092078DC02AF099
:1011D0008EC02BF08FC02CF090C02DF095C02EF05B
:1011E00096C02FF097C030F098C031F013ECACF0FF
:1011F000D8A0FDEF88F0FFEF88F0C8EF88F066C058
:1012000009F00A6ACAECB9F009500001826F82C085
:1012100081F0670E8219D8A410EF89F012EF89F0DF
:1012200038EF89F0ED51EE11D8A419EF89F01BEFDA
:1012300089F01FEF89F0000EEE6F010EED6FEEBF2B
:101240002CEF89F0EE5106E1ED05D8B02AEF89F0D8
:101250002CEF89F032EF89F0000E7E6F060E7D6F65
:1012600041EF89F0EDC07DF0EEC07EF041EF89F0F6
:10127000EEBF3DEF89F03FEF89F02CEF89F032EFC0
:1012800089F0670E8219D8A448EF89F04AEF89F0F7
:1012900079EF89F092AF58EF89F0FC0E915DFF0E67
:1012A0009259D8A056EF89F058EF89F077EF89F07E
:1012B000FF0E576EFF0E586E7DC059F07EC05AF07B
:1012C0005750592658505A229151595C5A50800A09
:1012D0005B6E9251800A5B58D8A071EF89F073EF72
:1012E00089F077EF89F0660E816F79EF89F0650EEE
:1012F000816F7DC073F07EC074F0670E8219D8A430
:1013000084EF89F086EF89F096EF89F0660E8119F7
:10131000D8A48DEF89F08FEF89F098EF89F092BF14
:1013200096EF89F094EF89F098EF89F0734B742B66
:10133000660E8119D8A49FEF89F0A1EF89F0C1EF63
:1013400089F092BFA8EF89F0A6EF89F0B4EF89F099
:10135000000E956F000E966F800E976F3F0E986F80
:10136000000E926F000E916F670E8219D8B4BBEF1A
:1013700089F0BDEF89F0C1EF89F091517327925147
:101380007423000E8C6F000E8B6F8DC083F08EC0A7
:1013900084F08FC085F090C086F095C075F096C03F
:1013A00076F097C077F098C078F052EF8AF083C05B
:1013B0002AF084C02BF085C02CF086C02DF095C09B
:1013C0002EF096C02FF097C030F098C031F0CAECE4
:1013D00097F02AC043F02BC044F02CC045F02DC03C
:1013E00046F0B9ECA1F043C087F044C088F045C096
:1013F00089F046C08AF087C003F088C004F089C035
:1014000005F08AC006F090ECABF003C079F004C0A0
:101410007AF083C02AF084C02BF085C02CF086C0FF
:101420002DF095C015F096C016F097C017F098C033
:1014300018F087C011F088C012F089C013F08AC07C
:1014400014F0A3EC95F011C02EF012C02FF013C0D1
:1014500030F014C031F0EDECB9F02AC083F02BC0AD
:1014600084F02CC085F02DC086F095C02AF096C07F
:101470002BF097C02CF098C02DF0000E2E6E000EB1
:101480002F6E200E306E410E316ECAEC97F02AC0DE
:1014900095F02BC096F02CC097F02DC098F000016D
:1014A0008B4B8C2B73518B5D8C51800A576E745112
:1014B000800A5758D8A05FEF8AF061EF8AF0D7EF23
:1014C00089F095C011F096C012F097C013F098C043
:1014D00014F0000E156E000E166EA00E176E400E64
:1014E000186EA3EC95F011C087F012C088F013C0FD
:1014F00089F014C08AF083C02AF084C02BF085C024
:101500002CF086C02DF087C02EF088C02FF089C047
:1015100030F08AC031F013ECACF0D8B092EF8AF022
:1015200094EF8AF09FEF8AF0000E0001876F000EA3
:10153000886F000E896F000E8A6FC8EF8AF083C033
:1015400003F084C004F085C005F086C006F087C0B3
:1015500007F088C008F089C009F08AC00AF087EC5B
:10156000B1F0D8A0B6EF8AF0B8EF8AF0C8EF8AF0F1
:10157000000179B1BEEF8AF0C0EF8AF0C8EF8AF0BF
:10158000000E876F000E886F000E896F000E8A6F45
:101590008DC003F08EC004F08FC005F090C006F03F
:1015A00087C007F088C008F089C009F08AC00AF037
:1015B00043EC93F003C083F004C084F005C085F0D1
:1015C00006C086F083C02AF084C02BF085C02CF0C2
:1015D00086C02DF0000E156E000E166E200E176ED2
:1015E000410E186E75C011F076C012F077C013F07E
:1015F00078C014F0A3EC95F011C02EF012C02FF0BB
:1016000013C030F014C031F013ECACF0D8A00BEFE5
:101610008BF00DEF8BF036EF8BF00001914B922B9E
:1016200075C011F076C012F077C013F078C014F0D6
:10163000000E156E000E166E200E176E410E186EFF
:10164000A3EC95F011C075F012C076F013C077F0DE
:1016500014C078F0660E00018119D8A432EF8BF027
:1016600034EF8BF036EF8BF0734B742B75C095F025
:1016700076C096F077C097F078C098F0650E0001BC
:101680008119D8B446EF8BF048EF8BF04EEF8BF01A
:1016900091C071F092C072F052EF8BF0000E726F39
:1016A000000E716F000E706F000E6F6F000E6E6F88
:1016B000000E6D6F000E8C6F000E8B6F4EEF8CF076
:1016C00083C02AF084C02BF085C02CF086C02DF09A
:1016D00095C02EF096C02FF097C030F098C031F032
:1016E000CAEC97F02AC043F02BC044F02CC045F060
:1016F0002DC046F0B9ECA1F043C087F044C088F09B
:1017000045C089F046C08AF087C003F088C004F065
:1017100089C005F08AC006F090ECABF003C079F008
:1017200004C07AF05CB897EF8BF099EF8BF0B7EFCD
:101730008BF0000179517A11D8A4A1EF8BF0A3EFBF
:101740008BF0B7EF8BF0670E8219D8A4AAEF8BF05D
:10175000ACEF8BF0B7EF8BF072BFB3EF8BF0B1EF64
:101760008BF0B7EF8BF06D4B6E2B02EF8CF000011E
:101770006F517011D8A4BFEF8BF0C1EF8BF0EBEF7E
:101780008BF072BFC8EF8BF0C6EF8BF0EBEF8BF0F6
:10179000200E9325D96E020E9421DA6E2E0EDF6E86
:1017A000934B942B7F07D8A08007000E706F010E1B
:1017B0006F6FEBEF8BF0200E9325D96E020E942104
:1017C000DA6E300EDF6E934B942B7F07D8A0800724
:1017D0006D07D8A06E076D516E11D8A4F2EF8BF093
:1017E000F4EF8BF0DBEF8BF0200E9325D96E020E19
:1017F0009421DA6E7951300FDF6E934B942B7F0773
:10180000D8A0800783C02AF084C02BF085C02CF0BC
:1018100086C02DF095C015F096C016F097C017F051
:1018200098C018F087C011F088C012F089C013F07A
:101830008AC014F0A3EC95F011C02EF012C02FF066
:1018400013C030F014C031F0EDECB9F02AC083F0D1
:101850002BC084F02CC085F02DC086F095C02AF0F6
:1018600096C02BF097C02CF098C02DF0000E2E6E75
:10187000000E2F6E200E306E410E316ECAEC97F0C6
:101880002AC095F02BC096F02CC097F02DC098F090
:1018900000017107D8A072078B4B8C2B73518B5DA5
:1018A0008C51800A576E7451800A5758D8B05BEF3C
:1018B0008CF05DEF8CF06BEF8CF094BF69EF8CF0E7
:1018C000945109E14B0E935DD8A069EF8CF06BEF5A
:1018D0008CF060EF8BF06F517011D8A472EF8CF028
:1018E00074EF8CF085EF8CF05CA879EF8CF07BEFD7
:1018F0008CF085EF8CF0200E9325D96E020E94218A
:10190000DA6E2E0EDF6E934B942B200E9325D96E3C
:10191000020E9421DA6E000EDF6E650E8119D8A4D6
:1019200094EF8CF096EF8CF0FCEF87F0000E8C6F4C
:101930004F0E8B6F200E8B25D96E020E8C21DA6E26
:10194000000EDF6E000E7C6F000E7B6F92BFADEF5E
:101950008CF0ABEF8CF0B5EF8CF0000E7C6F010ECD
:101960007B6F916D921FD8B0922B000E7E6F020E8E
:101970007D6FE6EF8CF08B07D8A08C07200E8B25AF
:10198000D96E020E8C21DA6E91C003F092C004F081
:10199000000E066E0A0E056ED8ECB0F00350300F44
:1019A000DF6E91C003F092C004F0000E066E0A0EC6
:1019B000056E15ECB0F003C091F004C092F0000188
:1019C0007D07D8A07E077F07D8A08007915192118C
:1019D000D8A4EDEF8CF0EFEF8CF0BBEF8CF07EBF76
:1019E000FCEF8CF07E5106E17D05D8B0FAEF8CF06B
:1019F000FCEF8CF0BBEF8CF08B07D8A08C077B51F1
:101A00007C11D8A406EF8DF008EF8DF00EEF8DF06D
:101A1000000E6A6F2B0E696F12EF8DF0000E6A6F69
:101A20002D0E696F200E8B25D96E020E8C21DA6E79
:101A30006000A7F1DFFF7F07D8A080078B07D8A041
:101A40008C07BF0E576EFF0E586E6651596E5A6A5C
:101A50005750592658505A225A5009E11A0E595CCB
:101A6000D8A035EF8DF037EF8DF03DEF8DF0000E03
:101A70006C6F650E6B6F41EF8DF0000E6C6F450E55
:101A80006B6F200E8B25D96E020E8C21DA6E6000F2
:101A9000AFF1DFFF7F07D8A08007200E9325076EE8
:101AA000020E9421086E200E8B25096E020E8C21E9
:101AB0000A6E1BECB7F0FCEF87F0120060006FF2CB
:101AC000D9FF600073F2DAFF6F007BFFF6FF6F0053
:101AD00077FFF7FF000EF86E0800F550250AD8A42E
:101AE00074EF8DF076EF8DF01FEF93F060006FF2E2
:101AF000D9FF600073F2DAFFDE2A000EDD22000E4D
:101B000001015D6F000E5C6F5CC15CF05DC15DF05A
:101B10000001ED69EE69000EAE6F000EAD6FDFEFF4
:101B20008DF05C8060006FF2D9FF600073F2DAFF25
:101B3000DE2A000EDD22DFEF8DF05C8292EF8DF069
:101B40005C8492EF8DF05C8692EF8DF05C8892EF72
:101B50008DF0000EAE6F010EAD6FDFEF8DF0600007
:101B60006FF2D9FF600073F2DAFF6F007BFFF6FFC0
:101B70006F0077FFF7FF000EF86E0800F5509F6FBB
:101B8000A06BA051000AD8B4C8EF8DF0A9EF8DF07A
:101B90009F51200AD8B4A3EF8DF0030AD8B4A6EF62
:101BA0008DF0080AD8B4A0EF8DF0060AD8B491EFF2
:101BB0008DF01D0AD8B49DEF8DF0A9EF8DF0AD51D9
:101BC000AE11D8B4E6EF8DF0E8EF8DF0AFEF8DF009
:101BD0005CA0EDEF8DF0EFEF8DF0F0EF8DF05C920B
:101BE00060006FF2D9FF600073F2DAFF6F007BFFD5
:101BF000F6FF6F0077FFF7FF000EF86E0800F55054
:101C00002A0AD8A406EF8EF008EF8EF03CEF8EF093
:101C100060006FF2D9FF600073F2DAFFDE2A000E77
:101C2000DD22600077F2D9FF60007BF2DAFF6F00FF
:101C30007CFF9FF0020EDE266F007CFFA0F0000EFE
:101C4000DD2260007FF2D9FF600083F2DAFF6F00CF
:101C500078FF5CF16F0074FF5DF101015DBF35EF4E
:101C60008EF033EF8EF07FEF8EF05C805C6D5D1F49
:101C7000D8B05D2B7FEF8EF060006FF2D9FF60006F
:101C800073F2DAFF6F0078FF0AF06F0074FF0BF059
:101C90001AECA7F00AC05CF10BC05DF159EF8EF0B1
:101CA00060006FF2D9FF600073F2DAFFDE2A000EE7
:101CB000DD22D00E00019F6FFF0EA06F60006FF25B
:101CC000D9FF600073F2DAFF6F007BFFF6FF6F0051
:101CD00077FFF7FF000EF86E0800F550A16FA26BBA
:101CE0009F51A127A051A223A25109E10A0EA15D93
:101CF000D8A07DEF8EF07FEF8EF050EF8EF0600079
:101D00006FF2D9FF600073F2DAFF6F007BFFF6FF1E
:101D10006F0077FFF7FF000EF86E0800F5502E0AEF
:101D2000D8A495EF8EF097EF8EF027EF8FF0000E8E
:101D30000001EE6F000EED6F60006FF2D9FF6000E2
:101D400073F2DAFFDE2A000EDD2260006FF2D9FFA7
:101D5000600073F2DAFF6F007BFFF6FF6F0077FF22
:101D6000F7FF000EF86E0800F5502A0AD8A4BBEF62
:101D70008EF0BDEF8EF0E4EF8EF060006FF2D9FFD1
:101D8000600073F2DAFFDE2A000EDD22600077F2D7
:101D9000D9FF60007BF2DAFF6F007CFF9FF0020E3C
:101DA000DE266F007CFFA0F0000EDD2260007FF2D7
:101DB000D9FF600083F2DAFF6F0078FFEDF06F006B
:101DC00074FFEEF027EF8FF060006FF2D9FF600034
:101DD00073F2DAFF6F0078FF0AF06F0074FF0BF008
:101DE0001AECA7F00AC0EDF00BC0EEF001EF8FF097
:101DF00060006FF2D9FF600073F2DAFFDE2A000E96
:101E0000DD22D00E00019F6FFF0EA06F60006FF209
:101E1000D9FF600073F2DAFF6F007BFFF6FF6F00FF
:101E200077FFF7FF000EF86E0800F550A16FA26B68
:101E30009F51A127A051A223A25109E10A0EA15D41
:101E4000D8A025EF8FF027EF8FF0F8EF8EF060002D
:101E50006FF2D9FF600073F2DAFF6F007BFFF6FFCD
:101E60006F0077FFF7FF000EF86E0800F550096E5F
:101E70000A6ACAECB9F009500001BD6FBD51D8B46F
:101E800044EF8FF046EF8FF090EF8FF060006FF22D
:101E9000D9FF600073F2DAFF6F0078FF9FF06F00E8
:101EA00074FFA0F0010E9F27000EA02360007FF2B8
:101EB000F6FF600083F2F7FF000EF86E0800F550A1
:101EC000096E0A6ACAECB9F009500001BE6FBE5132
:101ED000D8B46DEF8FF06FEF8FF090EF8FF0600060
:101EE0006FF2D9FF600073F2DAFF6F0078FF9FF0A6
:101EF0006F0074FFA0F0020E9F27000EA023600069
:101F00007FF2F6FF600083F2F7FF000EF86E080024
:101F1000F550096E0A6ACAECB9F009500001BF6FAA
:101F200060006FF2D9FF600073F2DAFF6F007BFF91
:101F3000F6FF6F0077FFF7FF000EF86E0800F55010
:101F4000630AD8A4A6EF8FF0A8EF8FF0D7EF8FF039
:101F500060006FF2D9FF600073F2DAFFDE2A000E34
:101F6000DD22600077F2D9FF60007BF2DAFF6F00BC
:101F70007CFF9FF0020EDE266F007CFFA0F0000EBB
:101F8000DD2260007FF2D9FF600083F2DAFFDF50CC
:101F9000C06F99C00CF09AC00DF0C0C00EF07AEC82
:101FA000AEF00CC099F00DC09AF042EF93F06000D3
:101FB0006FF2D9FF600073F2DAFF6F007BFFF6FF6C
:101FC0006F0077FFF7FF000EF86E0800F550640A07
:101FD000D8B4EDEF8FF0EFEF8FF007EF90F06000E7
:101FE0006FF2D9FF600073F2DAFF6F007BFFF6FF3C
:101FF0006F0077FFF7FF000EF86E0800F550690AD2
:10200000D8A405EF90F007EF90F051EF90F060004A
:102010006FF2D9FF600073F2DAFFDE2A000EDD22D4
:10202000600077F2D9FF60007BF2DAFF6F007CFF7F
:102030009FF0020EDE266F007CFFA0F0000EDD2276
:1020400060007FF2D9FF600083F2DAFF6F0078FF53
:10205000A3F06F0074FFA4F0000EA4BFFF0EA56FE5
:10206000A66FA76FA86FA96FAA6F99C01EF09AC03C
:102070001FF0A3C020F0A4C021F0A5C022F0A6C08C
:1020800023F0A7C024F0A8C025F0A9C026F0AAC05C
:1020900027F050EC9BF01EC099F01FC09AF042EF61
:1020A00093F0660EBD19D8A458EF90F05AEF90F057
:1020B000ADEF90F060006FF2D9FF600073F2DAFFCD
:1020C0006F007BFFF6FF6F0077FFF7FF000EF86EE3
:1020D00008006F00D4FFC0F060006FF2D9FF60000D
:1020E00073F2DAFFDE2A000EDD22600077F2D9FFFC
:1020F00060007BF2DAFF6F007CFF9FF0040EDE26AB
:102100006F007CFFA0F0000EDD2260007FF2D9FF9F
:10211000600083F2DAFF6F0078FFB9F06F0078FF9C
:10212000BAF06F0078FFBBF06F0078FFBCF099C089
:1021300060F09AC061F0B9C062F0BAC063F0BBC091
:1021400064F0BCC065F0C0C066F056EC87F060C0BB
:1021500099F061C09AF042EF93F0BD0E036E000E4D
:10216000046EFB0E056EFF0E066E000E086E020E6C
:10217000076E8BECA8F003500410D8A4C2EF90F0C7
:10218000C4EF90F058EF91F060006FF2D9FF60005B
:1021900073F2DAFF6F0078FF9FF06F0074FFA0F01A
:1021A000010E00019F27000EA02360007FF2F6FFC2
:1021B000600083F2F7FF000EF86E08006F00D4FF96
:1021C000C0F0BF0E9F6FFF0EA06F60006FF2D9FFCF
:1021D000600073F2DAFF6F007BFFF6FF6F0077FF9E
:1021E000F7FF000EF86E0800F550A16FA26B9F512B
:1021F000A127A051A223A25107E11A0EA15DD8B0D8
:1022000004EF91F006EF91F02AEF91F0600077F281
:10221000D9FF60007BF2DAFF6F007CFF9FF0040EB5
:10222000DE266F007CFFA0F0000EDD2260007FF252
:10223000D9FF600083F2DAFF6F0078FFB9F06F001A
:1022400078FFBAF06F0078FFBBF06F0078FFBCF04A
:102250004CEF91F0600077F2D9FF60007BF2DAFF7B
:102260006F007CFF9FF0040EDE266F007CFFA0F065
:10227000000EDD2260007FF2D9FF600083F2DAFFFA
:102280006F0078FFB9F06F0078FFBAF06F0078FF49
:10229000BBF06F0078FFBCF0020E60006FF2D9FF58
:1022A000600073F2DAFFDE26000EDD2297EF90F079
:1022B00060006FF2D9FF600073F2DAFF6F007BFFFE
:1022C000F6FF6F0077FFF7FF000EF86E0800F5507D
:1022D000730AD8B46EEF91F070EF91F08FEF91F038
:1022E00060006FF2D9FF600073F2DAFF6F0078FFD1
:1022F00003F06F0074FF04F0F30E056EFF0E066E20
:10230000000E086E030E076E8BECA8F0035004104D
:10231000D8A48DEF91F08FEF91F0E9EF91F060008C
:102320006FF2D9FF600073F2DAFF6F007BFFF6FFF8
:102330006F0077FFF7FF000EF86E0800F550730A84
:10234000D8B4A5EF91F0A7EF91F0AEEF91F0000EA9
:102350000001B06F030EAF6FB3EF91F0000E0001FC
:10236000B06F010EAF6F60006FF2D9FF600073F2C3
:10237000DAFFAF51DE26B051DD22600077F2D9FFDF
:1023800060007BF2DAFF6F007CFF9FF0020EDE261A
:102390006F007CFFA0F0000EDD2260007FF2D9FF0D
:1023A000600083F2DAFF6F0078FFABF06F0074FF1C
:1023B000ACF099C00CF09AC00DF0ABC00EF0ACC000
:1023C0000FF084ECA5F00CC099F00DC09AF042EF2C
:1023D00093F060006FF2D9FF600073F2DAFF6F00D4
:1023E0007BFFF6FF6F0077FFF7FF000EF86E080027
:1023F000F550750AD8A4FFEF91F001EF92F04DEF80
:1024000092F060006FF2D9FF600073F2DAFFDE2A0B
:10241000000EDD22600077F2D9FF60007BF2DAFF68
:102420006F007CFF9FF0020EDE266F007CFFA0F0A5
:10243000000EDD2260007FF2D9FF600083F2DAFF38
:102440006F0078FFA1F06F0074FFA2F0A1C0B1F09F
:10245000A2C0B2F00001B36BB46BB56BB66BB76BD7
:10246000B86B99C01EF09AC01FF0B1C020F0B2C086
:1024700021F0B3C022F0B4C023F0B5C024F0B6C040
:1024800025F0B7C026F0B8C027F0C2ECA2F01EC0FD
:1024900099F01FC09AF042EF93F060006FF2D9FFFD
:1024A000600073F2DAFF6F007BFFF6FF6F0077FFCB
:1024B000F7FF000EF86E0800F550780AD8B463EF05
:1024C00092F065EF92F07DEF92F060006FF2D9FF2D
:1024D000600073F2DAFF6F007BFFF6FF6F0077FF9B
:1024E000F7FF000EF86E0800F550580AD8A47BEFED
:1024F00092F07DEF92F0DDEF92F060006FF2D9FF85
:10250000600073F2DAFF6F007BFFF6FF6F0077FF6A
:10251000F7FF000EF86E08006F00D4FFC0F06000F7
:102520006FF2D9FF600073F2DAFFDE2A000EDD22BF
:10253000600077F2D9FF60007BF2DAFF6F007CFF6A
:102540009FF0020EDE266F007CFFA0F0000EDD2261
:1025500060007FF2D9FF600083F2DAFF6F0078FF3E
:10256000A1F06F0074FFA2F0A1C0B1F0A2C0B2F060
:102570000001B36BB46BB56BB66BB76BB86B99C03E
:102580001EF09AC01FF0B1C020F0B2C021F0B3C05D
:1025900022F0B4C023F0B5C024F0B6C025F0B7C017
:1025A00026F0B8C027F0C0C028F0C1EC9CF01EC0D7
:1025B00099F01FC09AF042EF93F060006FF2D9FFDC
:1025C000600073F2DAFF6F007BFFF6FF6F0077FFAA
:1025D000F7FF000EF86E0800F550250AD8A4F3EFB7
:1025E00092F0F5EF92F00FEF93F060006FF2D9FFE9
:1025F000600073F2DAFFDE2A000EDD22000E046EA8
:10260000250E036E99C005F09AC006F00EECAEF0F0
:10261000000E00019A6F010E996F42EF93F0600077
:102620006FF2D9FF600073F2DAFFDE2A000EDD22BE
:10263000000E00019A6F000E996F42EF93F0600058
:102640006FF2D9FF600073F2DAFF6F007BFFF6FFD5
:102650006F0077FFF7FF000EF86E0800F550036E6D
:10266000046A99C005F09AC006F00EECAEF0600066
:102670006FF2D9FF600073F2DAFFDE2A000EDD226E
:1026800008EF93F012000650800B0F6E06500624E0
:10269000116E05AE4EEF93F050EF93F051EF93F0C3
:1026A00011801150D8B457EF93F059EF93F06EEFBB
:1026B00093F01128D8A45FEF93F061EF93F069EFE6
:1026C00093F0000E036E000E046E000E056E000EF9
:1026D000066E058E000E066E76EF93F0000E036E0A
:1026E000000E046E000E056E000E066E0A50800B82
:1026F000106E0F501018D8B480EF93F082EF93F063
:1027000083EF93F00F8C0A500A24106E09AE8BEF02
:1027100093F08DEF93F08EEF93F010801050D8B4BB
:1027200094EF93F096EF93F0ABEF93F01028D8A4CA
:102730009CEF93F09EEF93F0A6EF93F0000E076EE0
:10274000000E086E000E096E000E0A6E098E000E55
:102750000A6EB3EF93F0000E076E000E086E000EC7
:10276000096E000E0A6E1150105CD8B0BAEF93F0EB
:10277000BCEF93F0E3EF93F00FACC1EF93F0C3EF36
:1027800093F0C5EF93F0800E0F1A11C012F010C035
:1027900011F012C010F003C012F007C003F012C015
:1027A00007F004C012F008C004F012C008F005C021
:1027B00012F009C005F012C009F006C012F00AC0FC
:1027C00006F012C00AF0000E126E115010C00BF08D
:1027D0000C6A0B5E000E0C5A0CBEF8EF93F00C5016
:1027E00009E11A0E0B5CD8A0F8EF93F0FAEF93F022
:1027F00031EF94F00350041005100610D8A403EF35
:1028000094F006EF94F0010E07EF94F0000E126EB4
:10281000000E036E000E046E000E056E000E066EB6
:1028200010C011F03AEF94F012A019EF94F01BEFE2
:1028300094F021EF94F0D89012300109126E23EF3A
:1028400094F0D890123203A028EF94F02AEF94F07D
:102850002BEF94F0128E0634063205320432033226
:10286000112A1050115CD8A038EF94F03AEF94F090
:1028700014EF94F00FBC3FEF94F041EF94F081EF30
:1028800094F01150D8A447EF94F049EF94F053EF2F
:1028900094F0000E036E000E046E000E056E000E26
:1028A000066EA2EF95F00750032608500422095047
:1028B00005220A50062206A060EF94F062EF94F021
:1028C0000EEF95F012A067EF94F069EF94F06FEFC0
:1028D00094F0D89012300109126E71EF94F0D890F4
:1028E000123203A076EF94F078EF94F079EF94F041
:1028F000128E06340632053204320332112A0EEFEC
:1029000095F00750035C08500458095005580650CC
:10291000800A0B6E0A50800A0B58D8B092EF94F0E0
:1029200094EF94F0BFEF94F00350075C0B6E0450EB
:1029300008580C6E055009580D6E06500A580E6E58
:10294000FF0E0B24036EFF0E0C20046EFF0E0D20F5
:10295000056EFF0E0E20066E800E0F1A126C1250BE
:10296000D8A4B5EF94F0B7EF94F0C7EF94F0010E50
:102970000326000E042205220622C7EF94F007501A
:10298000035E0850045A0950055A0A50065A03506B
:10299000041005100610D8A4D0EF94F0D2EF94F0F4
:1029A00007EF95F01250D8A4D8EF94F0DAEF94F036
:1029B00007EF95F0000E036E000E046E000E056E1C
:1029C000000E066EA2EF95F0D89003360436053659
:1029D000063612AEEEEF94F0F0EF94F0F1EF94F0D3
:1029E000038012A0F6EF94F0F8EF94F0FCEF94F06F
:1029F000D8801236FEEF94F0D89012361150D8B429
:102A000004EF95F006EF95F007EF95F0110605AE8F
:102A10000CEF95F00EEF95F0E4EF94F0000E106ED1
:102A200012AE15EF95F017EF95F02FEF95F012C05D
:102A30000BF07F0E0B16D8B420EF95F022EF95F037
:102A400026EF95F0010E106E2FEF95F003A02BEFFF
:102A500095F02DEF95F02FEF95F022EF95F01050B7
:102A6000D8B435EF95F037EF95F062EF95F0010EA1
:102A70000326000E04220522062206A042EF95F04E
:102A800044EF95F062EF95F003C00BF004C00CF03A
:102A900005C00DF006C00EF00E340E320D320C32B1
:102AA0000B320BC003F00CC004F00DC005F00EC0DB
:102AB00006F01128D8B45FEF95F061EF95F062EF62
:102AC00095F0112A1128D8B468EF95F06AEF95F0C7
:102AD00072EF95F01150D8A470EF95F072EF95F069
:102AE00084EF95F0000E036E000E046E000E056E6E
:102AF000000E066E1150D8A480EF95F082EF95F08D
:102B000084EF95F0000E0F6E11A089EF95F08BEF1A
:102B100095F08EEF95F0058E8FEF95F0059ED8908D
:102B20001130066E0FAE97EF95F099EF95F09AEF92
:102B300095F0068E03C003F004C004F005C005F054
:102B400006C006F012001450800B1D6E14501424A1
:102B5000236E13AEAEEF95F0B0EF95F0B1EF95F0B8
:102B600023802350D8B4B7EF95F0B9EF95F0CCEFB0
:102B700095F02328D8A4BFEF95F0C1EF95F0C9EFE9
:102B800095F0000E116E000E126E000E136E000E08
:102B9000146E138ED4EF95F0000E116E000E126EAF
:102BA000000E136E000E146E1850800B1D1A185074
:102BB00018241E6E17AEDFEF95F0E1EF95F0E2EF0F
:102BC00095F01E801E50D8B4E8EF95F0EAEF95F02E
:102BD000FDEF95F01E28D8A4F0EF95F0F2EF95F0F8
:102BE000FAEF95F0000E156E000E166E000E176EC1
:102BF000000E186E178E05EF96F0000E156E000E83
:102C0000166E000E176E000E186E1E50D8B40BEF25
:102C100096F00DEF96F015EF96F02350D8A413EF31
:102C200096F015EF96F01FEF96F0000E116E000E65
:102C3000126E000E136E000E146EC9EF97F017504F
:102C400011026F00CCFF28F06F00D0FF29F0285050
:102C50001F6E206A216A226A2950246E256A266A1C
:102C6000276A165012026F00CCFF28F06F00D0FFC9
:102C700029F028501F26000E20222122222229502E
:102C80002426000E252226222722155013026F002B
:102C9000CCFF28F06F00D0FF29F028501F26000E2F
:102CA00020222122222229502426000E25222622FB
:102CB000272221C022F020C021F01FC020F01F6A6F
:102CC000155012026F00CCFF28F06F00D0FF29F0E2
:102CD00028501F2629502022000E2122000E2222D9
:102CE000165011026F00CCFF28F06F00D0FF29F0C2
:102CF00028501F2629502022000E2122000E2222B9
:102D000021C022F020C021F01FC020F01F6A155002
:102D100011026F00CCFF28F06F00D0FF29F028507F
:102D20001F2629502022000E2122000E2222175099
:102D300012026F00CCFF28F06F00D0FF29F028505E
:102D4000242629502522000E2622000E2722165066
:102D500013026F00CCFF28F06F00D0FF29F028503D
:102D6000242629502522000E2622000E2722175045
:102D700013026F00CCFF28F06F00D0FF29F028501D
:102D8000196E29501A6E1B6A1C6A1BC01CF01AC0EF
:102D90001BF019C01AF0196A195024261A5025225E
:102DA0001B5026221C5027221FC019F020C01AF0E9
:102DB00021C01BF022C01CF0190EE4EF96F0D89051
:102DC0001C321B321A321932E82EDFEF96F01950FE
:102DD00024261A5025221B5026221C50272221C0AF
:102DE00022F020C021F01FC020F01F6A1E5023C017
:102DF00019F01A6A1926000E1A22820E1924286E5A
:102E0000FF0E1A20296E1AEF97F0D8902436253637
:102E10002636273622AE0FEF97F011EF97F012EF1C
:102E200097F02480D8901F36203621362236280687
:102E3000D8A0290626AE1FEF97F021EF97F005EFF7
:102E400097F0000E1E6E22AE28EF97F02AEF97F053
:102E50004EEF97F0FF0E1F14196EFF0E20141A6E1E
:102E6000FF0E21141B6E7F0E22141C6E19501A10B7
:102E70001B101C10D8B43FEF97F041EF97F045EFCF
:102E800097F0010E1E6E4EEF97F024A04AEF97F0D8
:102E90004CEF97F04EEF97F041EF97F01E50D8B4FB
:102EA00054EF97F056EF97F07AEF97F0010E242643
:102EB000000E25222622272227A061EF97F063EF3C
:102EC00097F07AEF97F024C019F025C01AF026C0C9
:102ED0001BF027C01CF01C341C321B321A32193272
:102EE00019C024F01AC025F01BC026F01CC027F022
:102EF000284A292A29BE85EF97F0295008E1282879
:102F0000D8A085EF97F087EF97F091EF97F0000E3C
:102F1000246E000E256E800E266E7F0E276EBFEF8C
:102F200097F029BE9EEF97F0295006E12804D8B00B
:102F30009CEF97F09EEF97F0AAEF97F0000E246EAB
:102F4000000E256E000E266E000E276E000E1D6E02
:102F5000BFEF97F028C023F0FF0E2416FF0E2516B2
:102F60007F0E2616000E271623A0B9EF97F0BBEFB1
:102F700097F0BCEF97F0268ED8902330276E1D5027
:102F8000271224C011F025C012F026C013F027C06C
:102F900014F012002D50800B3A6E2D502D24416EEE
:102FA0002CAED5EF97F0D7EF97F0D8EF97F04180A0
:102FB0004150D8B4DEEF97F0E0EF97F0F5EF97F0DF
:102FC0004128D8A4E6EF97F0E8EF97F0F0EF97F0FC
:102FD000000E2A6E000E2B6E000E2C6E000E2D6E53
:102FE0002C8E000E2D6EFDEF97F0000E2A6E000E57
:102FF0002B6E000E2C6E000E2D6E3150800B3A1A87
:1030000031503124426E30AE08EF98F00AEF98F05C
:103010000BEF98F042804250D8B411EF98F013EFC4
:1030200098F028EF98F04228D8A419EF98F01BEFF9
:1030300098F023EF98F0000E2E6E000E2F6E000E0B
:10304000306E000E316E308E000E316E30EF98F023
:10305000000E2E6E000E2F6E000E306E000E316EC2
:103060002E502F1030103110D8A439EF98F03BEFCC
:1030700098F053EF98F0000E2A6E000E2B6E000EA3
:103080002C6E000E2D6E800E2C127F0E2D123A50DB
:103090002D122AC02AF02BC02BF02CC02CF02DC0F2
:1030A0002DF096EF99F04150D8A459EF98F05BEFCE
:1030B00098F065EF98F0000E2A6E000E2B6E000E51
:1030C0002C6E000E2D6E96EF99F0425041C032F0FA
:1030D000336A325E000E335A7F0E32243B6E000E8E
:1030E00033203C6E2AC036F02BC037F02CC038F0AD
:1030F0002DC039F0000E2A6E000E2B6E000E2C6EC5
:10310000000E2D6E000E3D6E000E3E6E000E3F6EE8
:10311000000E406E000E426EC6EF98F04250D8B4DA
:1031200094EF98F096EF98F0ADEF98F0D89036368F
:10313000373638363936D8902A362B362C362D3657
:1031400040AEA5EF98F0A7EF98F0A8EF98F02A808E
:10315000D8903D363E363F3640362E50365C2F50A6
:1031600037583050385831503958D8A0BAEF98F005
:10317000BCEF98F0C5EF98F0408C2E50365E2F5083
:10318000375A3050385A3150395A422A190E42644F
:10319000CCEF98F0CEEF98F08EEF98F036503710D5
:1031A00038103910D8B4D7EF98F0D9EF98F0F1EF84
:1031B00098F03D80F1EF98F0D8902A362B362C36D7
:1031C0002D3640AEE6EF98F0E8EF98F0E9EF98F092
:1031D0002A80D8903D363E363F3640363B06D8A052
:1031E0003C062CAEF6EF98F0F8EF98F0DCEF98F094
:1031F000000E426E40AEFFEF98F001EF99F025EF20
:1032000099F0FF0E3D14326EFF0E3E14336EFF0E2A
:103210003F14346E7F0E4014356E3250331034102C
:103220003510D8B416EF99F018EF99F01CEF99F01B
:10323000010E426E25EF99F02AA021EF99F023EFBD
:1032400099F025EF99F018EF99F04250D8B42BEF90
:1032500099F02DEF99F051EF99F0010E2A26000E0A
:103260002B222C222D222DA038EF99F03AEF99F045
:1032700051EF99F02AC032F02BC033F02CC034F05B
:103280002DC035F03534353234323332323232C03B
:103290002AF033C02BF034C02CF035C02DF03B4A5F
:1032A0003C2A3CBE5CEF99F03C5008E13B28D8A09A
:1032B0005CEF99F05EEF99F069EF99F0000E3C6ECB
:1032C0003B68000E2A6E000E2B6E000E2C6E000E58
:1032D0002D6E3CBE76EF99F03C5006E13B04D8B031
:1032E00074EF99F076EF99F084EF99F0000E3C6E50
:1032F000000E3B6E000E2A6E000E2B6E000E2C6E22
:10330000000E2D6E000E3A6E3BC041F041A08BEFD7
:1033100099F08DEF99F090EF99F02C8E91EF99F054
:103320002C9ED89041302D6E47EF98F01200B90EC8
:10333000036EF90E046E39ECB8F0B40E0001EF6FB5
:10334000010EF06F000E0101B46F430EB56FB66948
:10335000400E0001FA6F030EFB6FEFC018F0F0C0D3
:1033600019F0FBC01AF01B6AFA51B0ECB7F0C70EA7
:10337000036EFA0E046E39ECB8F0050E0101B46F5D
:10338000000EB56F340EB66F400E0001FA6FB40E2A
:10339000EF6F010EF06F030EFB6FEFC018F0F0C07F
:1033A00019F0FBC01AF01B6AFA51B0ECB7F0250E09
:1033B000036EF90E046E39ECB8F0060E0101B46F1D
:1033C000800EB56F000EB66F400E0001FA6FB40E9E
:1033D000EF6F010EF06F030EFB6FEFC018F0F0C03F
:1033E00019F0FBC01AF01B6AFA51B0ECB7F0540E9A
:1033F000036EF80E046E39ECB8F0070E0101B46FDD
:10340000270EB56F100EB66F400E0001FA6FB40EA6
:10341000EF6F010EF06F030EFB6FEFC018F0F0C0FE
:1034200019F0FBC01AF01B6AFA51B0ECB7F0400E6D
:103430000001FA6F000E0101B46F000EB56FB40EFB
:103440000001EF6F010EF06F040E186EEFC019F05F
:10345000F0C01AF0000E1C6E030E1B6EFA518EECBB
:10346000B4F00101B4510001E36FE26B0101B55109
:103470000001E225FC6F0101000E0001E321FD6F58
:10348000700EC96F020ECA6F4D0ECB6FFC0ECC6F63
:10349000FCC0CDF0FDC0CEF0B7ECB8F0700E036EFE
:1034A000020E046EACECB6F0400E0001FA6F000E96
:1034B0000101B46F000EB56FB40E0001EF6F010E85
:1034C000F06F070E186EEFC019F0F0C01AF0000E82
:1034D0001C6E030E1B6EFA518EECB4F00101B45158
:1034E0000001E36FE26B0101B5510001E225FC6FC1
:1034F0000101000E0001E321FD6F170E156EB70EDE
:10350000166E510E176E3F0E186EFCC003F0FDC014
:1035100004F0056A066A000EAAECA4F003C011F0DC
:1035200004C012F005C013F006C014F0A3EC95F02F
:1035300011C02AF012C02BF013C02CF014C02DF0D3
:10354000000E2E6E000E2F6E000E306E470E316E86
:10355000CAEC97F02AC03AF12BC03BF12CC03CF1E9
:103560002DC03DF1700E0001C96F020ECA6FAC0E86
:10357000CB6FFB0ECC6F3AC1CDF03BC1CEF03CC15E
:10358000CFF03DC1D0F0B7ECB8F0700E036E020E74
:10359000046EACECB6F0400E0001FA6F000E0101B3
:1035A000B46F000EB56F000EB66FB40E0001EF6F72
:1035B000010EF06FFE0E186EEFC019F0F0C01AF099
:1035C000000E1C6E030E1B6EFA518EECB4F001015E
:1035D000B4510001E36FE26B0101B5510001E22536
:1035E000FC6F0101000E0001E321FD6F700EC96F39
:1035F000020ECA6FF90ECB6FFC0ECC6FFCC0CDF083
:10360000FDC0CEF0B7ECB8F0700E036E020E046E83
:10361000ACECB6F0400E0001FA6F000E0101B46F81
:10362000000EB56F000EB66FB40E0001EF6F010E05
:10363000F06FFF0E186EEFC019F0F0C01AF0000E18
:103640001C6E030E1B6EFA518EECB4F00101B451E6
:103650000001E36FE26B0101B5510001E225FC6F4F
:103660000101000E0001E321FD6F700EC96F020E13
:10367000CA6F480ECB6FFD0ECC6FFCC0CDF0FDC005
:10368000CEF0B7ECB8F0700E036E020E046EACEC28
:10369000B6F03B0E036EFB0E046E39ECB8F0120070
:1036A00020C038F021C039F022C03AF023C03BF0EE
:1036B00024C03CF025C03DF026C03EF027C03FF0BE
:1036C0003FBE65EF9BF068EF9BF0010E69EF9BF04A
:1036D000000E366E376A36503710D8B472EF9BF052
:1036E00074EF9BF084EF9BF03F1E3E1E3D1E3C1E80
:1036F0003B1E3A1E391E386C000E39223A223B22FC
:103700003C223D223E223F220001EEBF8AEF9BF089
:103710008CEF9BF08DEF9BF05C92EEBF9AEF9BF0ED
:10372000EE5106E1ED05D8B098EF9BF09AEF9BF0D3
:10373000A0EF9BF0000E336E010E326EA4EF9BF0F3
:10374000EDC032F0EEC033F05CC134F05DC135F055
:1037500036503710D8A4AFEF9BF0B1EF9BF0B8EF25
:103760009BF05CA4B6EF9BF0B8EF9BF0BBEF9BF037
:103770003406D8A03506000E416E4F0E406E000E86
:1037800002016F6F40EF9CF04006D8A04106200E6A
:103790004024D96E020E4120DA6E38C003F039C0E1
:1037A00004F03AC005F03BC006F03CC007F03DC055
:1037B00008F03EC009F03FC00AF00A0E0B6E000E82
:1037C0000C6E000E0D6E000E0E6E000E0F6E000ED3
:1037D000106E000E116E000E126ED9ECA7F003C031
:1037E00028F004C029F005C02AF006C02BF007C05D
:1037F0002CF008C02DF009C02EF00AC02FF028C010
:1038000015F02AC016F097ECBAF01550300FDF6EA5
:103810003206D8A033063406D8A0350638C003F0E7
:1038200039C004F03AC005F03BC006F03CC007F0D8
:103830003DC008F03EC009F03FC00AF00A0E0B6E12
:10384000000E0C6E000E0D6E000E0E6E000E0F6E52
:10385000000E106E000E116E000E126E56ECA6F0E9
:1038600003C038F004C039F005C03AF006C03BF0A0
:1038700007C03CF008C03DF009C03EF00AC03FF070
:1038800041BE4BEF9CF0415008E14004D8A04BEF03
:103890009CF04DEF9CF07DEF9CF0385039103A10C1
:1038A0003B103C103D103E103F10D8A45AEF9CF046
:1038B0005CEF9CF0C4EF9BF033BE69EF9CF033509B
:1038C00006E13204D8B067EF9CF069EF9CF0C4EFDA
:1038D0009BF035BE74EF9CF0355008E13404D8A05D
:1038E00074EF9CF076EF9CF07DEF9CF05CB27BEF88
:1038F0009CF07DEF9CF0C4EF9BF036503710D8A4BD
:1039000084EF9CF086EF9CF08DEF9CF05CA48BEF35
:103910009CF08DEF9CF0ACEF9CF04006D8A04106E7
:1039200036503710D8A497EF9CF099EF9CF09FEF9A
:103930009CF0000E316E2B0E306EA3EF9CF0000E4B
:10394000316E2D0E306E200E4024D96E020E4120B5
:10395000DA6E6000C3F0DFFF1EC013F01FC014F06A
:10396000200E4024156E020E4120166E34C017F052
:1039700035C018F077ECB0F013C01EF014C01FF083
:1039800012000001EEBFC7EF9CF0C9EF9CF0CAEF38
:103990009CF05C92EEBFD7EF9CF0EE5106E1ED0596
:1039A000D8B0D5EF9CF0D7EF9CF0DDEF9CF0000E87
:1039B000326E010E316EE1EF9CF0EDC031F0EEC0E1
:1039C00032F05CC133F05DC134F05CA8EAEF9CF0EA
:1039D000ECEF9CF0F0EF9CF0FE0E3326FF0E34224D
:1039E00020C035F021C036F022C037F023C038F0B7
:1039F00024C039F025C03AF026C03BF027C03CF087
:103A0000000E3E6E4F0E3D6E000E02016F6FA3EF73
:103A10009DF03D06D8A03E060F0E35143F6E406A5D
:103A200040BE1CEF9DF0405009E10A0E3F5CD8A05B
:103A30001CEF9DF01EEF9DF026EF9DF0570E3F24EA
:103A40003F6E000E4020406E2CEF9DF0300E3F2464
:103A50003F6E000E4020406EBF0E296EFF0E2A6E94
:103A600028502B6E2C6A29502B262A502C222C50A1
:103A700007E11A0E2B5CD8B040EF9DF042EF9DF0AD
:103A800065EF9DF09F0E296EFF0E2A6E200E3F10EF
:103A90002B6E000E40102C6E29502B262A502C2203
:103AA0002C5007E11A0E2B5CD8B059EF9DF05BEF5C
:103AB0009DF065EF9DF03FC009F040C00AF033EC87
:103AC000BAF009C03FF00AC040F0200E3D24D96E84
:103AD000020E3E20DA6E6000FFF0DFFF3106D8A054
:103AE00032063306D8A0340635C029F036C02AF095
:103AF00037C02BF038C02CF039C02DF03AC02EF072
:103B00003BC02FF03CC030F0050E90EF9DF0D890F8
:103B100030322F322E322D322C322B322A322932B1
:103B2000E82E87EF9DF029C035F02AC036F02BC073
:103B300037F02CC038F02DC039F02EC03AF02FC02D
:103B40003BF030C03CF03EBEAFEF9DF03E5009E18F
:103B5000020E3D5CD8A0AFEF9DF0B1EF9DF0E1EF1C
:103B60009DF0355036103710381039103A103B1090
:103B70003C10D8A4BEEF9DF0C0EF9DF009EF9DF082
:103B800032BECDEF9DF0325006E13104D8B0CBEF1C
:103B90009DF0CDEF9DF009EF9DF034BED8EF9DF084
:103BA000345008E13304D8A0D8EF9DF0DAEF9DF04F
:103BB000E1EF9DF05CB2DFEF9DF0E1EF9DF009EFEA
:103BC0009DF05CA8E6EF9DF0E8EF9DF0FFEF9DF023
:103BD0003D06D8A03E06200E3D24D96E020E3E20A2
:103BE000DA6E6000A3F0DFFF3D06D8A03E06200E8F
:103BF0003D24D96E020E3E20DA6E300EDF6E1EC0FE
:103C000013F01FC014F0200E3D24156E020E3E204E
:103C1000166E33C017F034C018F077ECB0F013C054
:103C20001EF014C01FF01200400E0001FA6F000ECB
:103C30000101B46F000EB56FB40E0001EF6F010EFD
:103C4000F06F020E186EEFC019F0F0C01AF0000EFF
:103C50001C6E030E1B6EFA518EECB4F00101B451D0
:103C6000446E436AB5514324706F000E4420716F57
:103C7000400E0001FA6F000E0101B46F000EB56F27
:103C8000B40E0001EF6F010EF06F010E186EEFC061
:103C900019F0F0C01AF0000E1C6E030E1B6EFA51E4
:103CA0008EECB4F00101B451446E436AB551432423
:103CB000726F000E4420736F400E0001FA6F000E09
:103CC0000101B46F000EB56FB40E0001EF6F010E6D
:103CD000F06F070E186EEFC019F0F0C01AF0000E6A
:103CE0001C6E030E1B6EFA518EECB4F00101B45140
:103CF000446E436AB55143240001FC6F0101000E7C
:103D000044200001FD6F170E156EB70E166E510E92
:103D1000176E3F0E186EFCC003F0FDC004F0056A7C
:103D2000066A000EAAECA4F003C011F004C012F061
:103D300005C013F006C014F0A3EC95F011C02AF0F2
:103D400012C02BF013C02CF014C02DF0000E2E6EFC
:103D5000000E2F6E000E306E470E316ECAEC97F0DB
:103D60002AC03AF12BC03BF12CC03CF12DC03DF1F3
:103D7000400E0001FA6F000E0101B46F000EB56F26
:103D8000B40E0001EF6F010EF06F060E186EEFC05B
:103D900019F0F0C01AF0000E1C6E020E1B6EFA51E4
:103DA0008EECB4F00101B451446E436AB551432422
:103DB0006C6F000E44206D6F6CC143F06DC144F018
:103DC000040E456ED89044324332452EE2EF9EF009
:103DD00043500F0BAB6FAB05D8A4F1EF9EF0F3EFA0
:103DE0009EF0F4EF9EF0BA98400E0001FA6F000EBC
:103DF0000101B46F000EB56FB40E0001EF6F010E3C
:103E0000F06F040E186EEFC019F0F0C01AF0000E3B
:103E10001C6E030E1B6EFA518EECB4F00101B4510E
:103E2000446E436AB55143246E6F000E44206F6F99
:103E3000400E0001FA6F000E0101B46F000EB56F65
:103E4000B40E0001EF6F010EF06F030E186EEFC09D
:103E500019F0F0C01AF0000E1C6E030E1B6EFA5122
:103E60008EECB4F00101B451446E436AB551432461
:103E70000001FC6F0101000E44200001FD6FFCC039
:103E800003F0FDC004F0056A066A000EAAECA4F077
:103E900003C02AF004C02BF005C02CF006C02DF0A2
:103EA000000E2E6E400E2F6E1C0E306E450E316EC3
:103EB000CAEC97F02AC046F12BC047F12CC048F15C
:103EC0002DC049F11200000E0001F36F030EF46FD4
:103ED0006000CFF3D9FF6000D3F3DAFF000EDF6E8E
:103EE0003D017599738F000E0001E76F020EE66FBA
:103EF000E6517FECBBF00009D8B481EF9FF083EF6F
:103F00009FF08DEFA0F00001E735E731E26FE63179
:103F1000FC6FE2C0FDF0F3C0C9F0F4C0CAF0460E79
:103F2000CB6FFA0ECC6FE6C0CDF0E7C0CEF0FCC090
:103F3000CFF0FDC0D0F0B7ECB8F02EEFA0F0F3C09A
:103F400011F0F4C012F0620E136EFD0E146EF1EC5F
:103F5000BCF085EFA0F0700E036E020E046E0E0E24
:103F6000056EFF0E066E3AECB6F0F3C003F0F4C037
:103F700004F00DECB8F003C0E4F004C0E5F000017B
:103F8000E451F325076EE551F421086E700E096EB9
:103F9000020E0A6E1BECB7F085EFA0F0F3C011F033
:103FA000F4C012F0FC0E136EFE0E146EF1ECBCF0B9
:103FB00085EFA0F0F3C011F0F4C012F0D70E136E2D
:103FC000FE0E146EF1ECBCF085EFA0F0F3C011F022
:103FD000F4C012F08C0E136EFF0E146EF1ECBCF0F8
:103FE00085EFA0F0F3C011F0F4C012F0320E136EA2
:103FF000FE0E146EF1ECBCF085EFA0F0F3C011F0F2
:10400000F4C012F05F0E136EFF0E146EF1ECBCF0F4
:1040100085EFA0F0F3C011F0F4C012F0C80E136EDB
:10402000FF0E146EF1ECBCF085EFA0F0F3C011F0C0
:10403000F4C012F0C20E136EFC0E146EF1ECBCF064
:1040400085EFA0F0F3C011F0F4C012F0A50E136ECE
:10405000FF0E146EF1ECBCF085EFA0F0FCC0E2F0B6
:10406000FDC0E3F00001E351000AD8B43AEFA0F03C
:1040700022EFA0F0E251200AD8B49FEF9FF0010A8E
:10408000D8B49FEF9FF0030AD8B49FEF9FF0010AC6
:10409000D8B49FEF9FF0040AD8B49FEF9FF00F0AA7
:1040A000D8B4ABEF9FF0010AD8B4ABEF9FF0030A8E
:1040B000D8B4ABEF9FF01D0AD8B4CEEF9FF00F0A33
:1040C000D8B4DAEF9FF0010AD8B4DAEF9FF0030A10
:1040D000D8B4DAEF9FF0010AD8B4DAEF9FF0070AFC
:1040E000D8B4E6EF9FF07C0AD8B4F2EF9FF0170A3D
:1040F000D8B4FEEF9FF03F0AD8B40AEFA0F0C80A88
:10410000D8B416EFA0F022EFA0F0F3C003F0F4C093
:1041100004F0ACECB6F02BECBCF0020E0001E6258E
:10412000E66F000EE721E76FE7BFA0EFA0F0E751D1
:1041300009E1FC0EE65DD8A0A0EFA0F0A2EFA0F090
:1041400078EF9FF03D01739F75892BECBCF03D012A
:10415000738F12002BECBCF0000E0001F36F030E06
:10416000F46FF3C0C9F0F4C0CAF0990ECB6FFF0E24
:10417000CC6F96C1CDF097C1CEF0ABC1CFF0D06B74
:10418000B7ECB8F0000E0201706F700E0001C96F3D
:10419000020ECA6FB00ECB6FFE0ECC6F72C1CDF0A7
:1041A00073C1CEF070C1CFF071C1D0F0B7ECB8F0F0
:1041B000F3C011F0F4C012F0700E136E020E146E04
:1041C000F1ECBCF0700E0001C96F020ECA6FBD0E9B
:1041D000CB6FFF0ECC6F6EC1CDF06FC1CEF0B7ECE0
:1041E000B8F0F3C011F0F4C012F0700E136E020EAE
:1041F000146EF1ECBCF0AE0E156E470E166EA10EED
:10420000176E3F0E186E70C103F071C104F0056A9D
:10421000066A000EAAECA4F003C011F004C012F06C
:1042200005C013F006C014F0A3EC95F011C02AF0FD
:1042300012C02BF013C02CF014C02DF0000E2E6E07
:10424000000E2F6E7A0E306E440E316ECAEC97F06F
:104250002AC03EF12BC03FF12CC040F12DC041F1EE
:10426000000E156E000E166E200E176E400E186EA4
:1042700072C103F073C104F0000E04BEFF0E056EA0
:10428000066E010EAAECA4F003C011F004C012F0F7
:1042900005C013F006C014F0A3EC95F011C02AF08D
:1042A00012C02BF013C02CF014C02DF0000E2E6E97
:1042B000500E2F6EC30E306E470E316ECAEC97F063
:1042C0002AC042F12BC043F12CC044F12DC045F16E
:1042D000700E0001C96F020ECA6F9C0ECB6FFE0EEE
:1042E000CC6F3EC1CDF03FC1CEF040C1CFF041C157
:1042F000D0F042C1D1F043C1D2F044C1D3F045C1A6
:10430000D4F0B7ECB8F0F3C011F0F4C012F0700EB6
:10431000136E020E146EF1ECBCF0700E0001C96F4A
:10432000020ECA6F940ECB6FFD0ECC6F46C1CDF05E
:1043300047C1CEF048C1CFF049C1D0F03AC1D1F069
:104340003BC1D2F03CC1D3F03DC1D4F0B7ECB8F0E2
:10435000F3C011F0F4C012F0700E136E020E146E62
:10436000F1ECBCF0F3C003F0F4C004F0ACECB6F038
:10437000120032C153F033C154F034C155F035C18D
:1043800056F043C053F044C054F045C055F046C009
:1043900056F0810E476EFF0E486E53C049F054C070
:1043A0004AF055C04BF056C04CF0180EDDEFA1F0AE
:1043B000D8904C324B324A324932E82ED8EFA1F035
:1043C00049504724516E000E4820526E52BEF2EF03
:1043D000A1F0525009E1170E515CD8A0F2EFA1F004
:1043E000F4EFA1F0FEEFA1F043C043F044C044F06D
:1043F00045C045F046C046F0C1EFA2F052BE03EF03
:10440000A2F005EFA2F075EFA2F051C047F0FF0E49
:10441000486EFF0E496E7F0E4A6E000E4B6E476669
:1044200014EFA2F01CEFA2F04B344B324A32493267
:104430004832472E0FEFA2F048C04DF049C04EF071
:104440004AC04FF04BC050F04D505314476E4E5081
:104450005414486E4F505514496E505056144A6EBD
:104460004750481049104A10D8A439EFA2F03BEF4A
:10447000A2F03DEFA2F0F4EFA1F053C047F054C01A
:1044800048F055C049F056C04AF0200E4DEFA2F05A
:10449000D8904A32493248324732E82E48EFA2F0EB
:1044A0004750481049104A10D8B459EFA2F05BEFBA
:1044B000A2F063EFA2F04D5053264E5054224F50BD
:1044C0005522505056224D1C476E4E1C486E4F1CB4
:1044D000496E501C4A6E4750531648505416495066
:1044E00055164A505616B9EFA2F053C047F054C0C3
:1044F00048F055C049F056C04AF0200E85EFA2F0B2
:10450000D8904A32493248324732E82E80EFA2F042
:104510004750481049104A10D8A491EFA2F093EFE9
:10452000A2F09DEFA2F0000E536E000E546E000E2E
:10453000556E000E566EB9EFA2F0D8905334476E08
:104540005434486E5534496E56344A6E47504810BC
:1045500049104A10D8B4AFEFA2F0B1EFA2F0B9EF12
:10456000A2F0000E536E000E546E800E556EBF0EFC
:10457000566E53C043F054C044F055C045F056C089
:1045800046F012000001EEBFC8EFA2F0CAEFA2F0A1
:10459000CBEFA2F05C92EEBFD8EFA2F0EE5106E1B5
:1045A000ED05D8B0D6EFA2F0D8EFA2F0DEEFA2F082
:1045B000000E316E010E306EE2EFA2F0EDC030F071
:1045C000EEC031F05CC132F05DC133F020C034F098
:1045D00021C035F022C036F023C037F024C038F0B7
:1045E00025C039F026C03AF027C03BF0000E3D6EE2
:1045F0004F0E3C6E000E02016F6F75EFA3F03C068C
:10460000D8A03D06200E3C24D96E020E3D20DA6E65
:1046100034C003F035C004F036C005F037C006F0F2
:1046200038C007F039C008F03AC009F03BC00AF0C2
:104630000A0E0B6E000E0C6E000E0D6E000E0E6E4E
:10464000000E0F6E000E106E000E116E000E126E38
:10465000E5ECAEF003C028F004C029F005C02AF054
:1046600006C02BF007C02CF008C02DF009C02EF0BA
:104670000AC02FF02850300FDF6E3006D8A0310668
:104680003206D8A0330634C003F035C004F036C07B
:1046900005F037C006F038C007F039C008F03AC05E
:1046A00009F03BC00AF00A0E0B6E000E0C6E000EF5
:1046B0000D6E000E0E6E000E0F6E000E106E000ED0
:1046C000116E000E126E96ECADF003C034F004C013
:1046D00035F005C036F006C037F007C038F008C026
:1046E00039F009C03AF00AC03BF03C503D10D8B454
:1046F0007CEFA3F07EEFA3F0AEEFA3F034503510C3
:1047000036103710381039103A103B10D8A48BEF00
:10471000A3F08DEFA3F0FFEFA2F031BE9AEFA3F06C
:10472000315006E13004D8B098EFA3F09AEFA3F02F
:10473000FFEFA2F033BEA5EFA3F0335008E132043F
:10474000D8A0A5EFA3F0A7EFA3F0AEEFA3F05CB263
:10475000ACEFA3F0AEEFA3F0FFEFA2F01EC013F09A
:104760001FC014F0200E3C24156E020E3D20166E64
:1047700032C017F033C018F077ECB0F013C01EF061
:1047800014C01FF012000001E46F91EFA4F0030EBB
:10479000E86FE769E7C003F0E8C004F099ECBBF00C
:1047A0001F0E0001E715E26F000EE815E36FE251FE
:1047B000E311D8A4DEEFA3F0E0EFA3F00CEFA4F038
:1047C000000E0201706FE7C003F0E8C004F0000EB5
:1047D000066E0A0E056E15ECB0F003C0E5F004C0DD
:1047E000E6F0700E0001C96F020ECA6F2E0ECB6F7D
:1047F000FD0ECC6FE5C0CDF0E6C0CEF08EECB8F08B
:1048000022C0CFF023C0D0F0B7ECB8F0700E036E2A
:10481000020E046EACECB6F0680E0001E26FE40E1E
:10482000E82EFED7E22FFCD700F00001E707D8A062
:10483000E807E8BF27EFA4F0E85107E1020EE75DC3
:10484000D8B025EFA4F027EFA4F0CAEFA3F0A7EFAC
:10485000A4F0000EE86F000EE76FE7C003F0E8C0B9
:1048600004F099ECBBF01F0E0001E715E26F000E9B
:10487000E815E36FE251E311D8A441EFA4F043EF50
:10488000A4F06FEFA4F0000E0201706FE7C003F018
:10489000E8C004F0000E066E0A0E056E15ECB0F0CE
:1048A00003C0E5F004C0E6F0700E0001C96F020E0F
:1048B000CA6F2F0ECB6FFF0ECC6FE5C0CDF0E6C0F8
:1048C000CEF08EECB8F022C0CFF023C0D0F0B7EC21
:1048D000B8F0700E036E020E046EACECB6F0680E0B
:1048E0000001E26FE40EE82EFED7E22FFCD700F0C5
:1048F0000001E74BE82BE8BF85EFA4F0040EE85D6C
:10490000D8A085EFA4F087EFA4F02DEFA4F0A7EFD7
:10491000A4F0000E046E000E036E99ECBBF0A7EF3E
:10492000A4F00001E451E26FE36BE351000AD8B454
:104930009CEFA4F089EFA4F0E251000AD8B4C7EFCD
:10494000A3F0010AD8B429EFA4F089EFA4F02BEC6E
:10495000BCF012000B6E0B50D8B4B1EFA4F0B3EF63
:10496000A4F0D5EFA4F006BEBAEFA4F0B8EFA4F01F
:10497000D5EFA4F003C007F004C008F005C009F0AB
:1049800006C00AF0071E081E091E0A1E072A000E8E
:10499000082209220A2207C00DF008C00EF009C043
:1049A0000FF00AC010F0DDEFA4F003C00DF004C05A
:1049B0000EF005C00FF006C010F0035004100510F3
:1049C0000610D8A4E6EFA4F0E8EFA4F0F2EFA4F00C
:1049D000000E036E000E046E000E056E000E066ED5
:1049E00083EFA5F0960E0C6EFCEFA4F00C2AD89085
:1049F00010320F320E320D32000E0D14076E000E03
:104A00000E14086E000E0F14096EFE0E10140A6EBE
:104A10000750081009100A10D8A411EFA5F013EFE1
:104A2000A5F0F6EFA4F021EFA5F00C2A010E0D265B
:104A3000000E0E220F221022D89010320F320E32AA
:104A40000D32000E0D14076E000E0E14086E000ECF
:104A50000F14096EFF0E10140A6E0750081009108B
:104A60000A10D8A436EFA5F038EFA5F015EFA5F0A1
:104A700040EFA5F00C06D8900D360E360F361036E6
:104A80000FBE45EFA5F047EFA5F04FEFA5F0020EE2
:104A90000C604DEFA5F04FEFA5F03AEFA5F00CB08C
:104AA00054EFA5F056EFA5F057EFA5F00F9ED89064
:104AB0000C320CC007F0086A096A0A6A07C00AF0DB
:104AC000096A086A076A07500D1208500E12095049
:104AD0000F120A5010120B50D8B471EFA5F073EFFB
:104AE000A5F07BEFA5F006BE7AEFA5F078EFA5F074
:104AF0007BEFA5F0108E0DC003F00EC004F00FC0C8
:104B000005F010C006F0120020EEE2F110EE11F0F8
:104B1000060E6F006FFFE3FFE806FBE20EC01CF01D
:104B20000FC01DF01C501D10D8A499EFA5F09BEFED
:104B3000A5F09FEFA5F0110E1C6E000E1D6E1CC09F
:104B400003F01DC004F00DECB8F003C020F004C069
:104B500021F0EDC01EF0EEC01FF01FBEB2EFA5F0B9
:104B6000B4EFA5F0C9EFA5F020501E5C1F50800ADD
:104B7000106E2150800A1058D8A0C1EFA5F0C3EFE5
:104B8000A5F0C5EFA5F0C9EFA5F01EC020F01FC02D
:104B900021F020C01EF021C01FF05CC11AF05DC1E1
:104BA0001BF05CB0D6EFA5F0D8EFA5F0F5EFA5F0BF
:104BB000E6EFA5F0000E046E200E036E0CC005F0AB
:104BC0000DC006F00EECAEF0204A212A1A50205CEF
:104BD0002150800A106E1B50800A1058D8A0F3EFA5
:104BE000A5F0F5EFA5F0DAEFA5F0000E196E000EB6
:104BF000186E1EEFA6F0600073F0F6FF600077F00D
:104C0000F7FF000EF86E1F0EF76403D00800F55092
:104C100007D06F00DBFFE9FF6F00DFFFEAFFEF5017
:104C2000106E1050036E046A0CC005F00DC006F043
:104C30000EECAEF01C4A1D2A184A192A1E50185CA8
:104C40001950800A106E1F50800A1058D8A02BEF00
:104C5000A6F02DEFA6F0FBEFA5F05CA032EFA6F0DA
:104C600034EFA6F051EFA6F042EFA6F0000E046E6E
:104C7000200E036E0CC005F00DC006F00EECAEF079
:104C8000204A212A1A50205C2150800A106E1B50A5
:104C9000800A1058D8A04FEFA6F051EFA6F036EFDB
:104CA000A6F020C00CF021C00DF01200000E146E12
:104CB00012BE5FEFA6F05DEFA6F071EFA6F0121E38
:104CC000111E101E0F1E0E1E0D1E0C1E0B6C000E54
:104CD0000C220D220E220F22102211221222010E6E
:104CE000146E0ABE78EFA6F076EFA6F08AEFA6F073
:104CF0000A1E091E081E071E061E051E041E036C42
:104D0000000E0422052206220722082209220A2276
:104D1000010E141A20EE15F0070EDE6AE806FDE219
:104D20000B500C100D100E100F101010111012104F
:104D3000D8B49DEFA6F09FEFA6F0F1EFA6F0010E1C
:104D4000136EADEFA6F0D8900B360C360D360E363E
:104D50000F36103611361236132A12AEB2EFA6F005
:104D6000B4EFA6F0A3EFA6F0D89015361636173696
:104D7000183619361A361B361C360B50035C0C508D
:104D800004580D5005580E5006580F500758105033
:104D900008581150095812500A58D8A0D2EFA6F05E
:104DA000D4EFA6F0E5EFA6F00B50035E0C50045ACA
:104DB0000D50055A0E50065A0F50075A1050085AF7
:104DC0001150095A12500A5A1580D89012321132D5
:104DD00010320F320E320D320C320B32132EB4EF72
:104DE000A6F01450D8B4F7EFA6F0F9EFA6F009EF4B
:104DF000A7F01C1E1B1E1A1E191E181E171E161E9B
:104E0000156C000E16221722182219221A221B22B4
:104E10001C2215C003F016C004F017C005F018C01E
:104E200006F019C007F01AC008F01BC009F01CC03A
:104E30000AF01200000E136E000E126E000E116EBC
:104E4000000E106E26EFA7F00A4A0B2A60002BF026
:104E5000F6FF60002FF0F7FF000EF86E0800F55027
:104E6000200AD8B436EFA7F038EFA7F024EFA7F068
:104E7000F70E0C6EFF0E0D6E60002BF0F6FF60005B
:104E80002FF0F7FF000EF86E0800F5500E6E0F6A57
:104E90000C500E260D500F220F5009E1050E0E5C2E
:104EA000D8A055EFA7F057EFA7F024EFA7F061EFD8
:104EB000A7F0000E116E010E106E0A4A0B2A9EEF2B
:104EC000A7F060002BF0F6FF60002FF0F7FF000E58
:104ED000F86E0800F5500C6E0D6A0D50000AD8B43B
:104EE00074EFA7F09EEFA7F00C502B0AD8B45DEF3B
:104EF000A7F0060AD8B459EFA7F09EEFA7F012C0AA
:104F000003F013C004F0000E066E0A0E056EB3EC3B
:104F1000BCF060002BF0F6FF60002FF0F7FF000EF2
:104F2000F86E0800F550035E000E045A300E03249C
:104F3000126E000E0420136E5DEFA7F0D00E0C6E03
:104F4000FF0E0D6E60002BF0F6FF60002FF0F7FFF4
:104F5000000EF86E0800F5500E6E0F6A0C500E260B
:104F60000D500F220F5009E10A0E0E5CD8A0BBEFC6
:104F7000A7F0BDEFA7F07FEFA7F010501110D8A455
:104F8000C4EFA7F0C6EFA7F0D4EFA7F012C00CF063
:104F900013C00DF00C1E0D1E0C4A0D2A0CC00AF099
:104FA0000DC00BF0D8EFA7F012C00AF013C00BF041
:104FB0001200000E146E0ABEE2EFA7F0E0EFA7F0B9
:104FC000F4EFA7F00A1E091E081E071E061E051E86
:104FD000041E036C000E042205220622072208226A
:104FE00009220A22010E146E12BEFBEFA7F0F9EFA0
:104FF000A7F00BEFA8F0121E111E101E0F1E0E1EA2
:105000000D1E0C1E0B6C000E0C220D220E220F2208
:105010001022112212220B500C100D100E100F1026
:10502000101011101210D8B418EFA8F01AEFA8F051
:1050300062EFA8F0010E136E28EFA8F0D8900B369F
:105040000C360D360E360F36103611361236132A40
:1050500012AE2DEFA8F02FEFA8F01EEFA8F00B5026
:10506000035C0C5004580D5005580E5006580F5054
:105070000758105008581150095812500A58D8A013
:1050800044EFA8F046EFA8F056EFA8F00B50035EEF
:105090000C50045A0D50055A0E50065A0F50075A1C
:1050A0001050085A1150095A12500A5AD890123208
:1050B000113210320F320E320D320C320B32132EEF
:1050C0002FEFA8F01450D8B468EFA8F06AEFA8F05A
:1050D0007AEFA8F00A1E091E081E071E061E051EEE
:1050E000041E036C000E0422052206220722082259
:1050F00009220A2203C003F004C004F005C005F031
:1051000006C006F007C007F008C008F009C009F0A3
:105110000AC00AF0120003C00AF004C00BF005C078
:105120000CF006C00DF00706D8A00806072806E117
:105130000828D8A49EEFA8F0A0EFA8F0ADEFA8F043
:10514000000E046E000E036E33EFA9F00A4A0B2A1C
:105150000C4A0D2A0706D8A0080660002BF0F6FFBF
:1051600060002FF0F7FF000EF86E1F0EF76403D0FB
:105170000800F55007D06F00DBFFE9FF6F00DFFF8D
:10518000EAFFEF500009D8B4C8EFA8F0CAEFA8F0C2
:105190000EEFA9F0600033F0F6FF600037F0F7FF84
:1051A000000EF86E0800F5500009D8B4DAEFA8F048
:1051B000DCEFA8F00EEFA9F007500810D8B4E3EF29
:1051C000A8F0E5EFA8F00EEFA9F0600033F0F6FFCD
:1051D000600037F0F7FF000EF86E08006F00D4FF94
:1051E00009F060002BF0F6FF60002FF0F7FF000ED3
:1051F000F86E1F0EF76403D00800F55007D06F005B
:10520000DBFFE9FF6F00DFFFEAFFEF500918D8B4BA
:105210000CEFA9F00EEFA9F0A6EFA8F060002BF0BC
:10522000F6FF60002FF0F7FF000EF86E1F0EF76418
:1052300003D00800F55007D06F00DBFFE9FF6F00D7
:10524000DFFFEAFFEF50096E600033F0F6FF600009
:1052500037F0F7FF000EF86E0800F550095C036E9A
:10526000046AD8A004061200400E4AECB4F0030E03
:10527000256E080E246E770EE82EFED7242EFCD75E
:10528000252EFAD700F0000E276E000E266E22049F
:105290002310D8A44EEFA9F050EFA9F058EFA9F0D1
:1052A000530E036EF50E046E39ECB8F02BECBCF027
:1052B000000E296E000E286E22042310D8A463EF7E
:1052C000A9F065EFA9F096EFA9F028502910D8B4FD
:1052D0006CEFA9F06EEFA9F096EFA9F0070E281475
:1052E000246E000E2914256E24502510D8A47BEFBF
:1052F000A9F07DEFA9F096EFA9F026C024F027C011
:1053000025F0D89024362536D89024362536D890E6
:1053100024362536530E2424036EF50E2520046E04
:1053200039ECB8F0264A272A2BECBCF0EB0E2824E7
:10533000F66EF30E2920F76EF86A000EF8220800C8
:10534000F55006ECB4F022042310D8A4AAEFA9F07B
:10535000ACEFA9F0BBEFA9F0EB0E2824F66EF30E2C
:105360002920F76EF86A000EF8220800F550A7EC25
:10537000B9F02BECBCF0284A292A295009E1400E4B
:10538000285CD8A0C6EFA9F0C8EFA9F05CEFA9F09F
:10539000800E4AECB4F0D00E246ECA0EE82EFED772
:1053A000242EFCD71200F70E036EFF0E046E39ECAC
:1053B000B8F0000E1F6E300E73ECB3F0680E236E63
:1053C000E40EE82EFED7232EFCD700D0320E3BECA5
:1053D000BDF0000E1F6E300E73ECB3F0150E236E91
:1053E000C60EE82EFED7232EFCD700D0330E3BECA2
:1053F000BDF0000E1F6E300E73ECB3F0150E236E71
:10540000C60EE82EFED7232EFCD700D0340E3BEC80
:10541000BDF0000E1F6E250E73ECB3F0150E236E5B
:10542000C60EE82EFED7232EFCD700D0350E3BEC5F
:10543000BDF0010E1F6E280E73ECB3F0150E236E37
:10544000C60EE82EFED7232EFCD700D0360E3BEC3E
:10545000BDF0010E1F6E080E73ECB3F0150E236E37
:10546000C60EE82EFED7232EFCD700D0370E3BEC1D
:10547000BDF0010E1F6E010E73ECB3F0030E246E2F
:10548000080E236E770EE82EFED7232EFCD7242E8F
:10549000FAD700F0380E3BECBDF0010E1F6E060E81
:1054A00073ECB3F0150E236EC60EE82EFED7232E36
:1054B000FCD700D0390E3BECBDF0010E1F6E0C0E78
:1054C00073ECB3F0150E236EC60EE82EFED7232E16
:1054D000FCD700D04F0E3BECBDF04B0E3BECBDF0CB
:1054E0001200B7ECBDF00009D8B479EFAAF07BEF59
:1054F000AAF0B7EFAAF088EFAAF00FECBEF003EF26
:10550000ABF065ECBEF003EFABF0000E03EFABF0D9
:1055100018C10EF019C10FF020EE09F102D89BEF6F
:10552000AAF00500FA6EDE50FD6EDE50FE6EDE5013
:10553000FF6EFA501200106E116A1150000AD8B4B2
:10554000A4EFAAF085EFAAF01050010AD8B485EFB5
:10555000AAF0030AD8B47DEFAAF0010AD8B481EF0B
:10556000AAF0070AD8B485EFAAF085EFAAF0ACEC50
:10557000BDF00009D8B4BFEFAAF0C1EFAAF002EF66
:10558000ABF001012951030B0009D8B4CAEFAAF00E
:10559000CCEFAAF0D8EFAAF0010E106E2951030B40
:1055A000116E1050115E29511118FC0B1118296F42
:1055B00060008FF4D9FF600093F4DAFFDF50126EC1
:1055C000234B242B2507D8A0260725512611D8A424
:1055D000ECEFAAF0EEEFAAF0F6EFAAF0D1ECB4F0FF
:1055E000106E1050146E156AFAEFAAF0000E156EC8
:1055F000030E146E14C013F0125022ECBEF01350C0
:1056000003EFABF0030E1200270E0001FA6F020E3B
:105610004AECB4F0090E0001E36F1E0EE26FE40ED7
:10562000E82EFED7E22FFCD7E32FFAD700F0010EC9
:10563000266E1C0E276EFE0E286E010E95ECACF049
:10564000000E0201706F700E0001C96F020ECA6F6A
:10565000EA0ECB6FFE0ECC6F96C1CDF097C1CEF0A7
:10566000B7ECB8F0010E276E700E286E020E296E90
:10567000020EC8ECBCF0000E0201706F700E00014B
:10568000C96F020ECA6F4F0ECB6FFF0ECC6F70C189
:10569000CDF071C1CEF072C1CFF073C1D0F0B7ECD4
:1056A000B8F0010E276E700E286E020E296E030EE2
:1056B000C8ECBCF0000E0201706F700E0001C96FE3
:1056C000020ECA6F060ECB6FFE0ECC6F3EC1CDF040
:1056D0003FC1CEF040C1CFF041C1D0F042C1D1F0C6
:1056E00043C1D2F044C1D3F045C1D4F0B7ECB8F017
:1056F0000101AB05D8A47FEFABF081EFABF086EFF3
:10570000ABF0410E0201826F4C0E836F010E276ECB
:10571000700E286E020E296E040EC8ECBCF012004A
:10572000053406340C6E0C50D8A499EFABF09BEF07
:10573000ABF0A5EFABF0000E036E000E046E000E92
:10574000056E000E066E12EFACF003C007F004C049
:1057500008F005C009F006C00AF0200EB5EFABF066
:10576000D8900A32093208320732E82EB0EFABF097
:1057700007500B6E058EFF0E0316FF0E0416FF0E6C
:105780000516000E0616960E0C5E0CBECCEFABF0A6
:10579000CAEFABF0E2EFABF00C50800A970FD8B035
:1057A000D4EFABF0D6EFABF0D8EFABF09BEFABF0B4
:1057B000D89006320532043203320C3ED8EFABF0FB
:1057C000FAEFABF01F0E0C64E8EFABF0EAEFABF0D2
:1057D000F2EFABF09BEFABF0D89003360436053612
:1057E00006360C060C50D8A4F8EFABF0FAEFABF08D
:1057F000ECEFABF00B50D8B400EFACF002EFACF034
:105800000AEFACF0061E051E041E036C000E0422F7
:105810000522062203C003F004C004F005C005F011
:1058200006C006F01200000E2A14326E000E2B1471
:10583000336E800E2C14346E7F0E2D14356E325064
:10584000331034103510D8A428EFACF02AEFACF0A8
:1058500032EFACF0000E2A6E000E2B6E000E2C6E96
:10586000000E2D6E000E2E14326E000E2F14336EAD
:10587000800E3014346E7F0E3114356E325033107A
:1058800034103510D8A447EFACF049EFACF051EF2D
:10589000ACF0000E2E6E000E2F6E000E306E000E5D
:1058A000316E2DAE56EFACF058EFACF061EFACF0CE
:1058B0002A6C2B1ED8B02B2A2C1ED8B02C2A800E76
:1058C0002D5631AE66EFACF068EFACF071EFACF096
:1058D0002E6C2F1ED8B02F2A301ED8B0302A800E42
:1058E0003156000E2A1A000E2B1A000E2C1A800EAA
:1058F0002D1A000E2E1A000E2F1A000E301A800ECE
:10590000311A2E502A5C2F502B5830502C583150C1
:105910002D58D8B08EEFACF090EFACF093EFACF028
:10592000D89094EFACF0D8801200456E27C003F0F9
:1059300028C004F00DECB8F003C043F004C044F0FC
:1059400044BEAEEFACF0445007E1150E435CD8B056
:10595000ACEFACF0AEEFACF016EFADF02E0E036E88
:10596000000E046E27C005F028C006F03AECB6F031
:10597000000E426E43500001FE5D296E4450FF59F7
:105980002A6E26502B6E2C6A29502B5C2C50800AD4
:105990002D6E2A50800A2D58D8A0D1EFACF0D3EF4D
:1059A000ACF0D5EFACF0010E266E4504D8A4DBEFC9
:1059B000ACF0DDEFACF0E1EFACF026507F0F4AEC3D
:1059C000B4F0020E4518D8A4E8EFACF0EAEFACF062
:1059D000EEEFACF02650BF0F4AECB4F0030E4518C2
:1059E000D8A4F5EFACF0F7EFACF0FBEFACF026503D
:1059F000930F4AECB4F0040E4518D8A402EFADF0B2
:105A000004EFADF008EFADF02650D30F4AECB4F040
:105A1000150E296EC60EE82EFED7292EFCD700D013
:105A20002E0E216E000E226E80ECB7F0120036C1F1
:105A30000DF037C10EF038C10FF039C110F003C0BE
:105A40000DF004C00EF005C00FF006C010F00DC040
:105A500007F00EC008F00FC009F010C00AF0180ED1
:105A600037EFADF0D8900A32093208320732E82E0B
:105A700032EFADF007500B6E0C6A0B500C10D8A42F
:105A800044EFADF046EFADF066EFADF0D8900D34D9
:105A9000076E0E34086E0F34096E10340A6E07500C
:105AA000081009100A10D8A458EFADF05AEFADF065
:105AB00060EFADF0000E046E020E036E95EFADF0D8
:105AC000000E046E030E036E95EFADF00B280C1064
:105AD000D8A46DEFADF06FEFADF091EFADF00DC06C
:105AE00007F00EC008F00FC009F010C00AF0090E50
:105AF000D8900736083609360A36E82E78EFADF02A
:105B00000750081009100A10D8B489EFADF08CEFD7
:105B1000ADF0010E8DEFADF0000E036E046A95EF4F
:105B2000ADF0000E046E040E036E120020EE13F0B2
:105B3000070EDE6AE806FDE20B500C100D100E1089
:105B40000F10101011101210D8B4A9EFADF0ABEF78
:105B5000ADF0FDEFADF0010E1B6EB9EFADF0D890DA
:105B60000B360C360D360E360F3610361136123611
:105B70001B2A12AEBEEFADF0C0EFADF0AFEFADF04F
:105B8000D890133614361536163617361836193699
:105B90001A360B50035C0C5004580D5005580E502B
:105BA00006580F50075810500858115009581250F5
:105BB0000A58D8A0DEEFADF0E0EFADF0F1EFADF0B8
:105BC0000B50035E0C50045A0D50055A0E50065AE5
:105BD0000F50075A1050085A1150095A12500A5AB9
:105BE0001380D8901232113210320F320E320D3231
:105BF0000C320B321B2EC0EFADF013C003F014C0FB
:105C000004F015C005F016C006F017C007F018C064
:105C100008F019C009F01AC00AF012000550061069
:105C2000D8B415EFAEF017EFAEF020EFAEF00550A0
:105C30000610D8A41EEFAEF020EFAEF025EFAEF0C8
:105C400003506CECBEF079EFAEF020EE09F0055099
:105C5000D9260650DA22DE50DE10D8B432EFAEF08C
:105C600034EFAEF04FEFAEF020EE09F00550D9263C
:105C70000650DA2210EE03F00550E1260650E2222B
:105C8000DE50E65CE650800A0B6EDE50800A0B5850
:105C9000D8B04DEFAEF04FEFAEF079EFAEF020EEB2
:105CA00003F00550D9260650DA226F0078FF07F07E
:105CB0006F0074FF08F0600017F0D9FF60001BF060
:105CC000DAFF6F0078FF09F06F0074FF0AF00750E9
:105CD0000924D96E08500A20DA6E60000FF0DFFF49
:105CE00020EE03F00550D9260650DA22DE2A000EF7
:105CF000DD22120001015C515D11D8A482EFAEF0EB
:105D000084EFAEF08AEFAEF05CC112F05DC113F02B
:105D100090EFAEF0FF0E5C25126EFF0E5D21136E4C
:105D20005CA095EFAEF097EFAEF0A0EFAEF00EC036
:105D300003F0046A0CC005F00DC006F00EECAEF0E6
:105D400013BEA5EFAEF0A7EFAEF0A9EFAEF0ADEF4A
:105D5000AEF0000E136E000E126E000E116E000EED
:105D6000106EBFEFAEF0000E046E200E036E0CC07E
:105D700005F00DC006F00EECAEF0104A112A1250DC
:105D8000105C1150800A0F6E1350800A0F58D8A073
:105D9000CCEFAEF0CEEFAEF0B3EFAEF05CB0D3EF41
:105DA000AEF0D5EFAEF0DEEFAEF00EC003F0046A59
:105DB0000CC005F00DC006F00EECAEF0010E102484
:105DC0000C6E000E11200D6E12000B500C100D10F9
:105DD0000E100F10101011101210D8B4F2EFAEF018
:105DE000F4EFAEF03CEFAFF0010E136E02EFAFF048
:105DF000D8900B360C360D360E360F36103611365F
:105E00001236132A12AE07EFAFF009EFAFF0F8EF3A
:105E1000AEF00B50035C0C5004580D5005580E505A
:105E200006580F5007581050085811500958125072
:105E30000A58D8A01EEFAFF020EFAFF030EFAFF070
:105E40000B50035E0C50045A0D50055A0E50065A62
:105E50000F50075A1050085A1150095A12500A5A36
:105E6000D8901232113210320F320E320D320C3203
:105E70000B32132E09EFAFF003C003F004C004F09F
:105E800005C005F006C006F007C007F008C008F01E
:105E900009C009F00AC00AF01200000EBA6EBB6811
:105EA000040EBC6EEF0EC26EC368A10EC46E000E6F
:105EB0003A01606F000E506F000E406F000E816F50
:105EC0005169FC0E416FC00E616F000E006F000E35
:105ED000016F000E026F000E036F000E046F000EC4
:105EE000086F000E096F000E0A6F000E0B6F000E98
:105EF0000C6F000E0D6F000E0E6F000E0F6F070E71
:105F0000426F000E526F180E626F436953696369E6
:105F1000446954696469080E846F000E476F000E6F
:105F2000466F000E456F000E576F000E566F000E45
:105F3000556F000E676F000E666F000E656F0D0ED9
:105F4000116F260E126F210E136F220E146F000EAA
:105F5000156F130E166F170EE56F130EE16F140E0B
:105F6000E26F1200270E0001FA6FEFEFAFF0800E24
:105F70004AECB4F0EE0E216EF60E226E4EECB5F049
:105F8000800E4AECB4F00DEFB0F0C00E4AECB4F065
:105F9000EE0E216EF60E226E4EECB5F0C00E4AECFF
:105FA000B4F00DEFB0F0940E4AECB4F0EE0E216EAA
:105FB000F60E226E4EECB5F0940E4AECB4F00DEFF6
:105FC000B0F0D40E4AECB4F0EE0E216EF60E226E56
:105FD0004EECB5F0D40E4AECB4F00DEFB0F026C0A4
:105FE00028F027C029F02950000AD8B4FAEFAFF002
:105FF0000DEFB0F02850010AD8B4B7EFAFF0030AA4
:10600000D8B4C5EFAFF0010AD8B4D3EFAFF0070AA8
:10601000D8B4E1EFAFF00DEFB0F0D00E286ECA0E9D
:10602000E82EFED7282EFCD71200000E086E06BE02
:106030001EEFB0F01CEFB0F024EFB0F0056C061EC0
:10604000D8B0062A010E086E04BE2BEFB0F029EF7F
:10605000B0F031EFB0F0036C041ED8B0042A010E8A
:10606000081A000E0A6E000E096E05500610D8B40C
:106070003CEFB0F03EEFB0F066EFB0F0010E076E0F
:1060800046EFB0F0D89005360636072A06AE4BEF3D
:10609000B0F04DEFB0F042EFB0F0D89009360A36CC
:1060A0000550035C06500458D8A059EFB0F05BEFE0
:1060B000B0F060EFB0F00550035E0650045A09805E
:1060C000D89006320532072E4DEFB0F00850D8B404
:1060D0006CEFB0F06EEFB0F072EFB0F0096C0A1E2A
:1060E000D8B00A2A09C003F00AC004F012005CA06C
:1060F0007CEFB0F07EEFB0F088EFB0F015C00CF0A0
:1061000016C00DF013C00EF014C00FF055ECBAF02D
:1061100018BE8DEFB0F08FEFB0F095EFB0F017C074
:106120001CF018C01DF099EFB0F0000E1D6E000EAF
:106130001C6E000E1B6E000E1A6EABEFB0F0000E60
:10614000046E200E036E13C005F014C006F00EECB2
:10615000AEF01A4A1B2A1C501A5C1B50800A196E9A
:106160001D50800A1958D8A0B8EFB0F0BAEFB0F0BF
:106170009FEFB0F05CB0BFEFB0F0C1EFB0F0CBEF8D
:10618000B0F015C00CF016C00DF013C00EF014C026
:106190000FF055ECBAF015C003F016C004F00DEC8A
:1061A000B8F01C500324136E1D500420146E12000E
:1061B000000E086E04BEE1EFB0F0DFEFB0F0E7EFE5
:1061C000B0F0036C041ED8B0042A010E086E06BE9F
:1061D000EEEFB0F0ECEFB0F0F2EFB0F0056C061EB1
:1061E000D8B0062A05500610D8B4F9EFB0F0FBEF8E
:1061F000B0F01FEFB1F0010E076E03EFB1F0D890D1
:1062000005360636072A06AE08EFB1F00AEFB1F000
:10621000FFEFB0F00550035C06500458D8A013EF10
:10622000B1F015EFB1F019EFB1F00550035E065073
:10623000045AD89006320532072E0AEFB1F0085002
:10624000D8B425EFB1F027EFB1F02BEFB1F0036C2C
:10625000041ED8B0042A03C003F004C004F01200E6
:10626000DC0EF66E7B0EF76E010EF86E00EEC0F2DD
:1062700010EE14F009006F00D7FFEEFFE550E1507B
:10628000F9E1260EF66E780EF76E010EF86E00EE4E
:10629000C8F110EE2FF009006F00D7FFEEFFE550B8
:1062A000E150F9E1D60EF66E7C0EF76E010EF86E37
:1062B00009006F00D4FFFEF009006F00D4FFFFF06B
:1062C00000EE00F310EE00F1EE6AE550E150FCE163
:1062D000E250FAE100EE00F2C00EEE6AE806FDE1DF
:1062E00000EE00F1C80EEE6AE806FDE100EEEDF00A
:1062F000110EEE6AE806FDE15D6A5C6A080ED56E75
:10630000000ED66E000ED76E000100EF80F0000E7A
:1063100003140B6E000E04140C6E800E05140D6E2B
:106320007F0E06140E6E0B500C100D100E10D8A41C
:106330009CEFB1F09EEFB1F0A6EFB1F0000E036E4E
:10634000000E046E000E056E000E066E000E0714A1
:106350000B6E000E08140C6E800E09140D6E7F0E6D
:106360000A140E6E0B500C100D100E10D8A4BBEFBB
:10637000B1F0BDEFB1F0C5EFB1F0000E076E000E49
:10638000086E000E096E000E0A6E075003180FE12A
:10639000085004180CE10950051809E10A500618C4
:1063A000D8B4D5EFB1F0D7EFB1F0DAEFB1F0D890C3
:1063B000DBEFB1F0D8801200266E270E0001FA6FD5
:1063C0002250236E246A2350FE5DFF51800A256E01
:1063D0002450800A2558D8B0F0EFB1F0F2EFB1F0B8
:1063E000F4EFB1F0FE05226E2604D8A4FAEFB1F066
:1063F000FCEFB1F000EFB2F022507F0F4AECB4F0A6
:10640000020E2618D8A407EFB2F009EFB2F00DEF94
:10641000B2F02250BF0F4AECB4F0030E2618D8A4F5
:1064200014EFB2F016EFB2F01AEFB2F02250930F61
:106430004AECB4F0040E2618D8A421EFB2F023EFF2
:10644000B2F027EFB2F02250D30F4AECB4F0D00EE6
:10645000236ECA0EE82EFED7232EFCD71200036E41
:10646000010E046E010129B738EFB2F03AEFB2F035
:106470007FEFB2F003C022F129952987FC0E29177E
:106480000F0E276F010E216FF40E206F2989D20E97
:10649000006F7C0E016F010E026F000E126F000E76
:1064A000136FD20E036F7C0E046F010E056F000E8A
:1064B000146F000E156FD20E066F7C0E076F010E63
:1064C000086F000E166F000E176FD20E096F7C0E4C
:1064D0000A6F010E0B6F000E186F000E196FCE0EB3
:1064E0000C6F7C0E0D6F010E0E6F000E1A6F000EFA
:1064F0001B6F41ECBEF042ECBCF0000E046E045089
:10650000120001012989A5EFB2F054ECBEF0080E8B
:10651000D2EFB2F054ECBEF0070ED2EFB2F00101B0
:10652000252927ECBEF0040ED2EFB2F0070E0101D0
:106530002719D8B49EEFB2F0A0EFB2F0A2EFB2F0FC
:1065400057ECBEF00F0ED2EFB2F012C10EF013C135
:106550000FF002D8B6EFB2F00500FA6E0051FD6EF2
:106560000151FE6E0251FF6EFA501200106E116A58
:106570001150000AD8B4BFEFB2F096EFB2F010504D
:10658000010AD8B496EFB2F0030AD8B48AEFB2F099
:10659000010AD8B485EFB2F0070AD8B48FEFB2F091
:0665A00096EFB2F01200BC
:1065A8003901A3A7DAEFB2F0DCEFB2F023EFB3F0D2
:1065B80093A7E1EFB2F0E3EFB2F023EFB3F06F008F
:1065C800A0F7B2F10D0E0101B219D8B4EEEFB2F096
:1065D800F0EFB2F0FCEFB2F00001F65109E1800EE5
:1065E800F55DD8A0FAEFB2F0FCEFB2F014EFB3F01B
:1065F800010E0101B36F800E0001F525D96E030E5F
:10660800F621DA6E000EDF6EF5C0A4F1F6C0A5F132
:10661800000EF66F000EF56F3901939723EFB3F074
:10662800800EF525D96E030EF621DA6E6000CBF6E2
:10663800DFFFF54BF62BF5C0A4F1F6C0A5F111006C
:10664800C2ECBDF00009D8A42CEFB3F02EEFB3F0E4
:1066580031EFB3F0040E72EFB3F001012951030BCF
:106668000009D8B43AEFB3F03CEFB3F048EFB3F019
:10667800010E126E2951030B136E1250135E29512D
:106688001318FC0B1318296F2507D8A026072551C6
:106698002611D8B452EFB3F054EFB3F062EFB3F071
:1066A80051ECBEF060008FF4D9FF600093F4DAFF7C
:1066B800DF6E0101234B242B2EEFB3F081ECB2F0F7
:1066C800146E51ECBEF060008FF4D9FF600093F4B3
:1066D800DAFFDF6E0101234B242B14501200216EC8
:1066E800270E0001FA6F2150F00B0C09226E22C010
:1066F8001DF0FA5187ECBCF02A0EE82EFED700D028
:106708002150F00B0809226E22C01DF00001FA5139
:1067180087ECBCF02A0EE82EFED700D01F04D8A4C0
:1067280098EFB3F09AEFB3F0BEEFB3F021C020F0CA
:106738000F0E20162038F00B0C09226E22C01DF017
:106748000001FA5187ECBCF02A0EE82EFED700D0E3
:1067580021C020F00F0E20162038F00B0809226EF9
:1067680022C01DF00001FA5187ECBCF02A0EE82E79
:10677800FED700D01200086E035004100510D8B4DC
:10678800C8EFB3F0CAEFB3F0EBEFB3F00850030D66
:10679800000EF324D96E010EF420DA6E60000FF0BB
:1067A800DEFF600013F0DEFF600017F0DEFF085028
:1067B800020D120EF324D96E010EF420DA6E600079
:1067C8001BF0DEFF60001FF0DDFF05EFB4F008509E
:1067D800030D000EF324D96E010EF420DA6ED20EEA
:1067E800DE6E7C0EDE6E010EDE6E0850020D120E9D
:1067F800F324D96E010EF420DA6E000EDE6E000E60
:10680800DD6E1200206E270E0001FA6F2050F00B8B
:106818000D09F96FF9C01DF0FA5187ECBCF02A0E8A
:10682800E82EFED700D02050F00B09090001F96FBF
:10683800F9C01DF0FA5187ECBCF02A0EE82EFED7FD
:1068480000D020C01FF00F0E1F161F38F00B0D09C7
:106858000001F96FF9C01DF0FA5187ECBCF02A0E5F
:10686800E82EFED700D020C01FF00F0E1F161F38CD
:10687800F00B09090001F96FF9C01DF0FA5187EC16
:10688800BCF02A0EE82EFED700D01200206E270E8C
:106898000001FA6F2050F00B0C09216E21C01DF089
:1068A800FA5187ECBCF02A0EE82EFED700D0205013
:1068B800F00B0809216E21C01DF00001FA5187EC88
:1068C800BCF06A0EE82EFED700D020C01FF00F0ED5
:1068D8001F161F38F00B0C09216E21C01DF0000196
:1068E800FA5187ECBCF06A0EE82EFED700D020C023
:1068F8001FF00F0E1F161F38F00B0809216E21C05C
:106908001DF00001FA5187ECBCF06A0EE82EFED7A4
:1069180000D012001D6E19C020F01AC021F01BC053
:106928001EF01CC01FF01D502FECB2F00009D8B4A7
:10693800A0EFB4F0A2EFB4F097EFB4F0B60E096E82
:10694800720E0A6E010E0B6E1E0E0C6E000E0D6E90
:1069580087ECBDF0180E036E000E046E000E066E76
:10696800010E056E29ECBDF0000E096E000E0A6ED0
:10697800000E0B6E000E0C6E000E0D6E79ECBDF065
:1069880031ECBEF09DECBCF0E806D8B4CEEFB4F024
:10699800D0EFB4F0C6EFB4F0120001012989E6EF98
:1069A800B4F054ECBEF0070E0FEFB5F00101252945
:1069B80027ECBEF0030E0FEFB5F057ECBEF00A0E51
:1069C8000FEFB5F012C10EF013C10FF002D8F7EFB8
:1069D800B4F00500FA6E0051FD6E0151FE6E0251D1
:1069E800FF6EFA501200106E116A1150000AD8B4E6
:1069F80000EFB5F0E1EFB4F01050010AD8B4E1EFC0
:106A0800B4F0030AD8B4D5EFB4F0060AD8B4DAEF74
:106A1800B4F0E1EFB4F012003901949BA49BC49444
:106A2800260E3A01126F3F013E9F3E9F000E3E6FB9
:106A3800030E3F6F000E3A6F000E396F000E386F6D
:106A4800350E0101C46F070EC56F000EC66F000E2C
:106A5800C76FC40E686F010E696F20EE02F06851AF
:106A6800D9266951DA22DF503F013D6F010120EE3E
:106A780001F06851D9266951DA22DF503F013C6F95
:106A88006000A3F5D9FF6000A7F5DAFFDF503B6F80
:106A98003E8F1200000E256E000E246E68EFB5F0D2
:106AA800600087F0F6FF60008BF0F7FF000EF86ECD
:106AB8000800F55006ECB4F0214A222A244A252A77
:106AC800850EE82EFED700F0600087F0F6FF600024
:106AD8008BF0F7FF000EF86E0800F5500009D8B4E7
:106AE80078EFB5F07AEFB5F08AEFB5F00001FE5116
:106AF800245C2550800A236EFF51800A2358D8A0B1
:106B080088EFB5F08AEFB5F054EFB5F0120039010F
:106B1800A3A791EFB5F093EFB5F096EFB5F06F003E
:106B2800A0F7B2F1000E046E000E036E800E03246F
:106B3800D96E030E0420DA6E000EDF6E034A042AB3
:106B4800045009E17F0E035CD8A0ADEFB5F0AFEFBC
:106B5800B5F09AEFB5F0000E0101B36F3D01F2896F
:106B6800000EF96F000EFA6F000E0301806F000E21
:106B78000101A56F000EA46F000EB26F3901938D4D
:106B88009387120041ECBEF0020E0101286FD9EF85
:106B9800B5F00FECBEF000EFB6F065ECBEF000EF1C
:106BA800B6F000ECBEF000EFB6F014C10EF015C15F
:106BB8000FF020EE03F102D8ECEFB5F00500FA6E05
:106BC800DE50FD6EDE50FE6EDE50FF6EFA50120093
:106BD800106E116A1150000AD8B4F5EFB5F0D5EF70
:106BE800B5F01050020AD8B4CDEFB5F0010AD8B408
:106BF800D1EFB5F0D5EFB5F01200C3C0C7F0C4C0EF
:106C0800C8F0000E01015B6F000E5A6F23EFB6F05B
:106C1800C1C099F0C2C09AF0C70E00019B6F000E68
:106C28009C6FC5C09DF0C6C09EF05EEC8DF0000163
:106C3800995101015A2700019A5101015B23600013
:106C48001FF3F6FF600023F3F7FF000EF86E08004D
:106C5800F5500009D8A433EFB6F035EFB6F00CEFD5
:106C6800B6F05AC1C1F05BC1C2F01200600017F063
:106C7800F6FF60001BF0F7FF000EF86E08006F00CB
:106C8800D4FFB1F161EFB6F0600017F0F6FF6000D5
:106C98001BF0F7FF000EF86E08006F00D4FFB1F18B
:106CA80060000FF0D9FF600013F0DAFF6000C7F64C
:106CB800DFFF034A042A054A062A0101B151D8A474
:106CC80068EFB6F06AEFB6F048EFB6F060000FF084
:106CD800D9FF600013F0DAFF000EDF6E120032EC0D
:106CE800B9F001012951030B0009D8B47EEFB6F0C1
:106CF80080EFB6F08DEFB6F0B7ECBDF00009D8B470
:106D080088EFB6F08AEFB6F08DEFB6F0100E0101FD
:106D1800276F01012751030D2B0EF324F66EF40E95
:106D2800F420F76EF86A000EF82202D8A9EFB6F040
:106D38000500FA6E0900F550FD6E0900F550FE6E6B
:106D48000900F550FF6EFA5012000101276F12007A
:106D5800000E066E000E056ED5EFB6F03901A3A938
:106D6800B8EFB6F0BAEFB6F0B2EFB6F005500324BC
:106D7800D96E06500420DA6EDF503D01EA6F054AED
:106D8800062A06BED1EFB6F0065009E1810E055C71
:106D9800D8A0D1EFB6F0D3EFB6F0D5EFB6F0E3EF69
:106DA800B6F005500324D96E06500420DA6EDF5081
:106DB800D8A4E1EFB6F0E3EFB6F0B2EFB6F0120008
:106DC800FC0E01012917020E286F2995F3EFB6F082
:106DD80063ECBEF01AEFB7F00F0E1AEFB7F016C15A
:106DE8000EF017C10FF020EE06F102D806EFB7F04B
:106DF8000500FA6EDE50FD6EDE50FE6EDE50FF6E50
:106E0800FA501200106E116A1150000AD8B40FEF30
:106E1800B7F0F0EFB6F01050020AD8B4ECEFB6F0C5
:106E2800010AD8B4ECEFB6F0F0EFB6F0120009C0E2
:106E38000DF00AC00EF007C00FF008C010F00D509A
:106E48000B6E0E500C6E0D4A0E2A60002FF0F6FFE6
:106E5800600033F0F7FF000EF86E60003FF0D9FFD6
:106E6800600043F0DAFF0F4A102A1F0EF76403D0C0
:106E78000800F55007D06F00DBFFE9FF6F00DFFF68
:106E8800EAFFEF50DF6EDF50D8A44DEFB7F04FEFB9
:106E9800B7F023EFB7F01200D28AD2BE56EFB7F0A0
:106EA80059EFB7F0010E5AEFB7F0000E036ED29EFD
:106EB800D29CD28A550ED46EAA0ED46ED490000EEF
:106EC800D76E000ED66E080ED56E550ED46EAA0E6D
:106ED800D46ED48039018387828F81818491839F86
:106EE800849587918991809FD28CD28E03B002D0ED
:106EF800D29E01D0D28E1200000E256E000E246E96
:106F080091EFB7F024502124D96E25502220DA6E53
:106F1800DF5006ECB4F0244A252A24502124D96EE7
:106F280025502220DA6EDF50D8B49DEFB7F09FEFDE
:106F3800B7F0AFEFB7F00001FE51245C2550800A8E
:106F4800236EFF51800A2358D8A0ADEFB7F0AFEFFA
:106F5800B7F086EFB7F012001C6E1C502FECB2F0A1
:106F68000009D8B4BAEFB7F0BCEFB7F0B1EFB7F09B
:106F780018C003F019C004F01AC005F01BC006F0D1
:106F880029ECBDF0000E096E000E0A6E000E0B6EA5
:106F9800000E0C6E000E0D6E79ECBDF031ECBEF0FB
:106FA8009DECBCF0E806D8B4DCEFB7F0DEEFB7F044
:106FB800D4EFB7F012003901A3A1E5EFB7F0E7EF7E
:106FC800B7F0E9EFB7F00CEFB8F0A2AFEEEFB7F01B
:106FD800F0EFB7F0F2EFB7F00CEFB8F03D0179A59C
:106FE800F8EFB7F0FAEFB7F0FCEFB7F00CEFB8F046
:106FF80079AF01EFB8F003EFB8F005EFB8F00CEF98
:10700800B8F076A90AEFB8F00CEFB8F0DFEFB7F0F8
:10701800120003C005F004C006F015EFB8F0034AEB
:10702800042A60000FF0F6FF600013F0F7FF000E6F
:10703800F86E1F0EF76403D00800F55007D06F00F4
:10704800DBFFE9FF6F00DFFFEAFFEF500009D8A47C
:1070580030EFB8F032EFB8F013EFB8F00550035C3A
:10706800036E06500458046E120051EFB8F039014F
:10707800A3A941EFB8F043EFB8F03BEFB8F06000D8
:107088000FF0F6FF600013F0F7FF000EF86E08002F
:107098006F00D7FFEAFD034A042A60000FF0F6FFED
:1070A800600013F0F7FF000EF86E0800F5500009B5
:1070B800D8A461EFB8F063EFB8F03BEFB8F0120076
:1070C800066E000E0101616F000E606F7BEFB8F075
:1070D800520E046E2B0E036E000EE82EFED7032E02
:1070E800FCD7042EFAD700D00101604B612B065063
:1070F800036E046A0350605D6151800A056E045096
:10710800800A0558D8A08BEFB8F08DEFB8F06CEF77
:10711800B8F01200400E0001FA6F000E0101B46FC2
:10712800000EB56FB40E0001EF6F010EF06F040E84
:10713800186EEFC019F0F0C01AF0000E1C6E030EA6
:107148001B6EFA518EECB4F00101B451256E246A1D
:10715800B55124246E6F000E25206F6F6EC122F08A
:107168006FC123F01200CD0E0001D56F000ED66F4F
:10717800C9C0D7F0CAC0D8F0000EDB6F000EDA6FB6
:10718800000EE16F000EE06FD70EC16F000EC26FE8
:10719800CBC0C3F0CCC0C4F0D50EC56F000EC66F0F
:1071A80001ECB6F00001DA51C925D96EDB51CA21CC
:1071B800DA6E000EDF6E1200010E096E200E031843
:1071C8000410D8B4EAEFB8F0ECEFB8F005EFB9F076
:1071D800F70E056EFF0E066E03C007F004C008F038
:1071E8000550072606500822085009E1050E075CDD
:1071F800D8A001EFB9F003EFB9F005EFB9F0000E30
:10720800096E09C003F0046A1200166E010E176EAB
:10721800010129B512EFB9F014EFB9F030EFB9F068
:107228002985000E176E255127ECBEF01650D8B4EC
:1072380020EFB9F022EFB9F029EFB9F0040E0101FF
:10724800276F59ECBCF02EEFB9F0030E0101276F40
:10725800A1ECBDF05BECBDF017501200E3ECBDF003
:107268000009D8B43AEFB9F03CEFB9F040EFB9F003
:1072780060ECBEF05AEFB9F0CDECBDF00009D8B41F
:1072880048EFB9F04AEFB9F04EEFB9F05AECBEF05A
:107298005AEFB9F0D8ECBDF00009D8B456EFB9F000
:1072A80058EFB9F05AEFB9F05DECBEF0120020EEDD
:1072B80002F00E50D9260F50DA226F0078FF03F043
:1072C8006F0074FF04F060003BF0D9FF60003FF0EE
:1072D800DAFF6F0078FF05F06F0074FF06F029EC05
:1072E800BDF0000E096E000E0A6E000E0B6E000E49
:1072F8000C6E000E0D6E87ECBDF0020E1200000E33
:107308003D01EC6F000EED6F000EEE6F000EEF6F9B
:10731800000EF06F000EF16FB00EF26F800EF36F7B
:10732800000EF46F8A0EF56F000EF66F000EF76F01
:10733800000EF86F000EF96F000EFA6FF28BF289EB
:10734800390193971200046E800E056EC1EFB9F0F3
:10735800045005140009D8B4B4EFB9F0B6EFB9F089
:10736800BBEFB9F02A0E3BECBDF0BEEFB9F0200E32
:107378003BECBDF0D8900530056E0550D8A4C7EF9A
:10738800B9F0C9EFB9F0ACEFB9F01200BF0E0B6E4F
:10739800FF0E0C6E09C00DF00AC00EF00B500D2642
:1073A8000C500E220E5007E11A0E0D5CD8B0DFEF1C
:1073B800B9F0E1EFB9F0E8EFB9F0200E0910096E65
:1073C8000A500A6EECEFB9F009C009F00AC00AF0D9
:1073D8001200000E2E1A000E2F1A000E301A800E00
:1073E800311A2AC003F02BC004F02CC005F02DC0C0
:1073F80006F02EC007F02FC008F030C009F031C0E9
:107408000AF043EC93F003C02AF004C02BF005C047
:107418002CF006C02DF012003A0157A116EFBAF071
:1074280018EFBAF02AEFBAF02A0E3D01EA6F410EC2
:107438004BECBDF04C0E4BECBDF070ECBCF0010118
:107448008C4B8D2B3F013E8FF2ECBAF03901A09F97
:10745800000E3A01576FCB503901A19111009F0ED0
:107468000B6EFF0E0C6E09C00DF00AC00EF00B502B
:107478000D260C500E220E5007E11A0E0D5CD8B0E6
:1074880048EFBAF04AEFBAF050EFBAF05F0E0914BD
:10749800096E0A6A54EFBAF009C009F00AC00AF086
:1074A8001200000E126E000E116E66EFBAF010C0D8
:1074B80003F0046A0EC005F00FC006F00EECAEF043
:1074C800114A122A11500C24D96E12500D20DA6E6E
:1074D800DF50106E1050D8A474EFBAF076EFBAF0FF
:1074E8005BEFBAF01200000EAC6E010EAE6E000E2D
:1074F8000101EA6F030EE96FE9C103F0033AAC50EA
:1075080003188F0B0318AC6E0F0EAC12FA0EAB6E8D
:10751800080EAF6E000E856F000E846F39019495CA
:10752800A495AC8E120016BEA4EFBAF0165006E170
:107538001504D8B0A2EFBAF0A4EFBAF0B2EFBAF0DF
:1075480015C017F016C018F0171E181E174A182A6B
:1075580017C015F018C016F0B6EFBAF015C015F040
:1075680016C016F012009F0E056EFF0E066E200E56
:107578000310076E000E0410086E0550072606500B
:10758800082208500AE11A0E075CD8A0CEEFBAF01C
:10759800D1EFBAF0010ED2EFBAF0000E036E046A12
:1075A8001200000EA06E050EA26E700EA0120F0E35
:1075B800A012F40E9F6E000E9E6E000EA36E000EBB
:1075C80001017B6F000E7A6F000E816F000E806FD5
:1075D800A79939019781A791A08E1200000EA06E7D
:1075E800050EA26E700EA0120F0EA012F40E9F6E62
:1075F800000E9E6E000EA36E000E01017B6F000E42
:107608007A6F000E816F000E806FA79939019781FC
:10761800A791A08E12009F0E056EFF0E066E03C086
:1076280007F004C008F00550072606500822085045
:107638000AE11A0E075CD8A024EFBBF027EFBBF0D5
:10764800010E28EFBBF0000E036E046A1200BF0E95
:10765800056EFF0E066E03C007F004C008F0055063
:1076680007260650082208500AE11A0E075CD8A01F
:1076780040EFBBF043EFBBF0010E44EFBBF0000E50
:10768800036E046A12000350041005100610D8B4E3
:1076980050EFBBF052EFBBF05AEFBBF0000E031AED
:1076A800000E041A000E051A800E061A03C003F015
:1076B80004C004F005C005F006C006F01200D00EA4
:1076C800056EFF0E066E03C007F004C008F00550F3
:1076D80007260650082208500AE10A0E075CD8A0BF
:1076E80078EFBBF07BEFBBF0010E7CEFBBF0000E38
:1076F800036E046A1200036E3D01799560000FF075
:107708006EFD000E6C6F738B79A58DEFBBF08FEF5C
:10771800BBF088EFBBF074AB94EFBBF097EFBBF016
:10772800010E98EFBBF0000E120003C005F004C074
:1077380006F0D89006320532D89006320532055048
:107748006D6E03C005F0030E0516060E066ED89082
:107758000536062EABEFBBF005506C6E12000EC05E
:1077680003F00FC004F0000E066E010E056E29EC42
:10777800BDF0000E096E000E0A6E000E0B6E000EB4
:107788000C6E000E0D6E87ECBDF0040E12000EC0DC
:1077980003F00FC004F0000E066E020E056E29EC11
:1077A800BDF0000E096E000E0A6E000E0B6E000E84
:1077B8000C6E000E0D6E87ECBDF0020E12000EC0AE
:1077C80003F00FC004F0000E066E010E056E29ECE2
:1077D800BDF0000E096E000E0A6E000E0B6E000E54
:1077E8000C6E000E0D6E87ECBDF0020E12000EC07E
:1077F80003F00FC004F0000E066E020E056E29ECB1
:10780800BDF0000E096E000E0A6E000E0B6E000E23
:107818000C6E000E0D6E87ECBDF0040E1200000019
:10782800007D803E401FA00FD007E803F40118F741
:1078380003F70EF7C4F6D9F6286E756C6C290003A9
:0D7848000001000200040008001000008094
:107856003901A3A931EFBCF033EFBCF02BEFBCF03C
:107866000D0E3D01EA6F3901A3A93CEFBCF03EEFD6
:10787600BCF036EFBCF00A0E3D01EA6F12003D0186
:1078860073BF48EFBCF04AEFBCF058EFBCF0000EF7
:10789600796F000E7A6F000E766F6C69510E3A01A1
:1078A6006A6F510E6B6F3D01738F120001012951F2
:1078B600FC0B0209296F25052611D8A465EFBCF03B
:1078C60067EFBCF069EFBCF081ECB2F0D880010143
:1078D600223522ECBEF0040E12003901A3A976EF80
:1078E600BCF078EFBCF070EFBCF00D0E3D01EA6F16
:1078F6003901A3A981EFBCF083EFBCF07BEFBCF0AC
:107906000A0E3D01EA6F12001E6E1DC0B4F1000E94
:107916000101B56FB40E186E010E196E000E1B6EC6
:10792600010E1A6E1E50B0ECB7F0A00E00D0E82E75
:10793600FDD71200010E036E010129B5A5EFBCF0BB
:10794600A7EFBCF0B1EFBCF02997226941ECBEF07D
:107956006AECBDF01CECBEF028C103F00350120027
:10796600035005026F00CCFF07F06F00D0FF08F050
:1079760003500602F350082604500502F350082669
:1079860007C003F008C004F012002B6E27C022F0D7
:107996002B50DCECB1F028C021F029C022F080EC9D
:1079A600B7F0150E2A6EC60EE82EFED72A2EFCD785
:1079B60000D0120048ECBEF045ECBEF00009D8B489
:1079C600E7EFBCF0E9EFBCF0EFEFBCF0000E27EC00
:1079D600BEF0000E22ECBEF0000E120011C003F045
:1079E60012C004F00DECB8F003501124076E0450D9
:1079F6001220086E13C009F014C00AF01BECB7F091
:107A060012006F0060FF02F0000E0101816F010E8F
:107A1600806F3F013E9FBA88A09E39019791A7913A
:107A260060000BF0D8FF1100030E3D017B6F040EC2
:107A3600736F800E746F000E756F000E6C6F759904
:107A46006000EBF36EFD7995739F1200010129A981
:107A56002FEFBDF031EFBDF03AEFBDF003C023F1DB
:107A660004C024F105C025F106C026F129991200AB
:107A7600036E3FEFBDF000F03901A3A945EFBDF05D
:107A860047EFBDF03EEFBDF060000FF0EAFD1200DB
:107A9600016E4FEFBDF000F03901A3A955EFBDF01F
:107AA60057EFBDF04EEFBDF0600007F0EAFD1200A3
:107AB60061EFBDF0DFECB7F073ECB6F0010129B56C
:107AC60067EFBDF069EFBDF05DEFBDF01200390163
:107AD60093939395929F93913D017A917A957A9F8C
:107AE6007A9D7A93769376957691120009C003F083
:107AF6000AC004F00BC005F00CC006F00DC007F07C
:107B0600020EBFECB3F0120009C003F00AC004F085
:107B16000BC005F00CC006F00DC007F0000EBFEC60
:107B2600B3F01200800E6E6E000E6D6E000E6C6E5F
:107B36003F015F51FC0B01095F6F120001012951E2
:107B4600FC0B0209296F2251222522ECBEF0030EFE
:107B560012003D0178BBB2EFBDF0B5EFBDF0010EEE
:107B6600B6EFBDF0000E12003D0174BBBDEFBDF0D7
:107B7600C0EFBDF0010EC1EFBDF0000E12003D01D9
:107B860078B1C8EFBDF0CBEFBDF0010ECCEFBDF084
:107B9600000E12003D0179B5D3EFBDF0D6EFBDF072
:107BA600010ED7EFBDF0000E12003D0176B9DEEFF3
:107BB600BDF0E1EFBDF0010EE2EFBDF0000E1200E8
:107BC6003D0179BFE9EFBDF0ECEFBDF0010EEDEF41
:107BD600BDF0000E12000FF584F438F6A5F686F611
:107BE60093F561F6CAF4CDF505F62CECBEF001016D
:107BF6002995020E286F0F0E12002CECBEF0010123
:107C06002995000E286F0F0E12004BECBEF048ECC3
:107C1600BEF016ECBEF012000101255127ECBEF0B5
:107C260059ECBCF0120001012995000E286F0F0EC9
:107C360012003D01739F000E796F78851200036E66
:107C460060000FF06BFD1200036E60000FF06CFD1C
:107C560012003D01739F7885738F1200000E09ECA8
:107C6600B9F012004BECBEF0090E12004EECBEF05D
:107C7600040E12004EECBEF0030E1200000E3D0183
:107C8600796F12003D016C5112003D01739B120089
:107C96003D01748D12003D01749D12003D016A5133
:107CA60012003D01738D12003D01739D12003D01CE
:107CB600799512003D01769912003D01799F1200D7
:107CC600010E1200020E1200050E1200010E120025
:047CD6001400120084
:020000040030CA
:0A0000008CD5FFF78DCFFFDFFFFF67
:00000001FF
